:1000000000800020BD010000E1590000AD59000052
:10001000AD590000AD590000AD590000AD590000C8
:10002000AD590000AD590000AD590000E159000084
:10003000E1590000AD590000E15900009D59000050
:10004000E1590000E1590000E1590000E1590000C8
:10005000E1590000E1590000E1590000E1590000B8
:10006000E1590000E1590000E1590000E1590000A8
:10007000E1590000E1590000E1590000E159000098
:10008000E1590000E1590000E1590000E159000088
:10009000E1590000E1590000E1590000E159000078
:1000A000E1590000E1590000E1590000E159000068
:1000B000E1590000E1590000E1590000E159000058
:1000C000E1590000E1590000E1590000E159000048
:1000D000E1590000E1590000E1590000E159000038
:1000E000E1590000E1590000E1590000E159000028
:1000F000E15900003D660000E1590000FD6B000081
:10010000E1590000D9700000E1590000E1590000F8
:10011000E1590000E1590000E1590000E1590000F7
:10012000E159000015080000450B0000E1590000EE
:10013000E1590000E1590000E1590000E1590000D7
:10014000E1590000E1590000E1590000E1590000C7
:10015000158000002D800000458000005D800000BB
:10016000E1590000E1730000E1590000E15900008D
:10017000E1590000E1590000E1590000E159000097
:10018000E1590000E1590000E159000099510000D7
:10019000E1590000E1590000E1590000E159000077
:1001A000E1590000E1590000E1590000E159000067
:1001B000E1590000E1590000E1590000564B4CF2B2
:1001C000205210B51A804DF628121A8000BF00BFC9
:1001D00005F00AFC514B4FF010621A60504A9A60C9
:1001E000504ADA60A3F53043203B1A6812F480725B
:1001F00004D14D490A604FF4A8521A604B4B1A784B
:10020000110703D51A7842F008021A70484B2A22C7
:100210001A700023474A48499818884204D247492F
:10022000595899500433F5E7454A464B9A424FF0E6
:10023000000302D242F8043BF7E74349434A5958C6
:1002400099500433B3F5DE7FF7D1414B802103F899
:10025000011B40498B42F9D13F4B1A603F4B0A22A8
:100260001A70A3F5805324225A70A0221A709A792A
:100270009207FCD59A79D406FCD4394B9A7902F0CE
:100280000C02082AF9D103221A7140225A719A7974
:100290009006FCD5324B9A795106FBD5314A32494A
:1002A00011600221516020221A702D4B9B7903F0BE
:1002B0000C030C2BF9D12D4B2D4A1A602D4B2E4AD5
:1002C0001A6000225A60072243F8042C2B4AC3F814
:1002D0000C2D62B605F01EFF134B1B68DA0705D51F
:1002E000274805F03BFD274B274A1A60274B1B7810
:1002F0005B0609D5234C244A2368934204D1204845
:1003000005F02CFD0023236008F038FC05F072FB9B
:1003100007F061FFFEE700BF0E200540308004407B
:10032000823F04000100002B14D0034002D007409C
:1003300000E007406087FF1F8088FF1F44BF000068
:100340008088FF1F0892FF1F000000000082FF1F2F
:1003500000E400E05FE400E008ED00E0005006404B
:100360000040064044800440000003010480044033
:10037000C010050014E000E0FF760100000020201E
:1003800000DD68501CE00340A5C3945A00F007400C
:10039000FFFFFFFFFFFFFFFFFFFFFFFFFFFFFFFF6D
:1003A000FFFFFFFFFFFFFFFFFFFFFFFFFFFFFFFF5D
:1003B000FFFFFFFFFFFFFFFFFFFFFFFFFFFFFFFF4D
:1003C000FFFFFFFFFFFFFFFFFFFFFFFFFFFFFFFF3D
:1003D000FFFFFFFFFFFFFFFFFFFFFFFFFFFFFFFF2D
:1003E000FFFFFFFFFFFFFFFFFFFFFFFFFFFFFFFF1D
:1003F000FFFFFFFFFFFFFFFFFFFFFFFFFFFFFFFF0D
:10040000FFFFFFFFFFFFFFFFFFFFFFFFFEFFFFFFFD
:1004100010B5054C237833B9044B13B10448AFF33E
:1004200000800123237010BD8088FF1F00000000A2
:1004300044BF000008B5064B1BB106480649AFF3A0
:1004400000800648036813B1054B03B1984708BD07
:100450000000000044BF00008488FF1F8088FF1F49
:10046000000000002DE9F04101210D2005F01EFDE6
:100470006D4B6E4C6E4E20221A604FF4887007F060
:10048000B2FE054602F02CFC2846256002F0ADFBCA
:10049000FE2811D140F2DC5005F026FE902007F036
:1004A000A2FE644904464FF4E13201F095F834604D
:1004B000306802F05DF9FBE723685F4993F8AA0012
:1004C00005F05CFC5D4B4FF496721A605C4BC022E9
:1004D0001A602368012193F8AA0005F0E7FC23685D
:1004E000402193F8AA0005F0FDFC0C2005F034F83B
:1004F000082005F05BF840F2DC5005F0F5FD2068BF
:1005000002F035FB430803F1376303F5D833B3FB3F
:10051000F0F005F04DFE206802F04BFB20B123689F
:1005200093F8A80005F0E8FE206802F04CFB4308B1
:1005300003F1376303F5D833B3FBF0F006F010F99D
:10054000206802F049FB430803F1B76303F5584301
:10055000B3FBF0F006F0E6FB206802F034FB054642
:10056000582007F040FE2A463649374D074603F02B
:10057000F3FE20682F6002F0FAFA80466C2007F044
:1005800032FE42463149074603F054FA304B5820B8
:100590001F6007F028FE074600F086FC2D4B2E4911
:1005A0001F60384600F0ECFD902007F01CFE21494A
:1005B0004FF4E132074601F00FF82068376002F08F
:1005C0000BFB0746902007F00EFE3A4622490646EE
:1005D00001F002F8214B28681E6003F025FF28680F
:1005E0001F4E03681B6A98473768286807F2FD2783
:1005F00003F0E2FE3368BB4204D2286803681B6A3A
:100600009847F7E760210B4620680A4602F073FA24
:1006100000F0DAF823681B7E23B10120BDE8F04129
:1006200004F0BCBCBDE8F08184F00F40B888FF1F27
:100630009C88FF1FD091FF1F0000A041A888FF1FCA
:10064000A088FF1F9891FF1FC088FF1F8891FF1F80
:10065000B488FF1FB088FF1FA891FF1FBC88FF1F31
:10066000D489FF1F1C4B1A684FF6E85101328A42A9
:1006700070B51A601D462EDD184C2368D3F8B400FF
:1006800004F00AF923680C2690FBF6F6986804F04B
:10069000F9F8B0F5967F05DDB0F5167FA8BF4FF4E9
:1006A000167001E04FF496700D4A23681268A0F5A9
:1006B00096700A21414391FBF2F10A4A93F8AA008D
:1006C0001268514301F52071F6B291FBF6F105F085
:1006D00009FC00232B6070BDAC88FF1FB888FF1F8A
:1006E000A888FF1FA088FF1F0F4B1A68002A08DA8E
:1006F0000E49086801280DD00120086020200C490F
:1007000007E007D00949086820B1002008600949BE
:100710002020086001324FF6E8518A42C8BF6FF0CE
:1007200031021A60704700BFA488FF1F6487FF1F53
:1007300084F00F4088F00F402DE9F0411D4F1E4D11
:100740003B681E4C93F8C430DFF878801C4E93B998
:10075000286802F00DF8206802F00AF8D8F80000C6
:1007600003F0C6FB306803681B6A9847FFF77AFFFF
:10077000FFF7BAFFE2E7D8F8000010B103689B6802
:100780009847306810B103689B689847286810B193
:1007900003689B689847206810B103689B68984776
:1007A00000F02EF83B681B7E0BB104F065FD00F0F5
:1007B00049FAFCE7B888FF1F9C88FF1FBC88FF1F11
:1007C000C088FF1FB488FF1F08B5094B4FF00072A7
:1007D0001A604FF080621A60064B1B6893F8250080
:1007E000054B187004F07CFF044B01221A7008BD01
:1007F00004E100E0B888FF1FC488FF1FC688FF1F00
:10080000034B4FF000721A604FF080621A6070471D
:1008100084E100E070B5B24C23780F2B00F28781A1
:10082000DFE813F0210036004B00600075008A00FD
:100830009F00B400C900DE001D0134010101680100
:100840004A011000A74D287804F092FFA64B1B68C0
:10085000D3F8B420132101FB0200142690FBF6F21A
:10086000C3F8B420D8E09F4D287804F081FF9E4B58
:100870001B681A6B452101FB0200462690FBF6F22D
:100880001A6393F82500287004F02AFF01234CE135
:10089000944D287804F06CFF934B1B685A6B4521EC
:1008A00001FB0200462690FBF6F25A6393F82600FD
:1008B000287004F015FF022337E18A4D287804F0F0
:1008C00057FF894B1B689A6B452101FB02004626A6
:1008D00090FBF6F29A6393F82700287004F000FF6B
:1008E000032322E17F4D287804F042FF7E4B1B68F2
:1008F000DA6B452101FB0200462690FBF6F2DA6333
:1009000093F82800287004F0EBFE04230DE1754DE8
:10091000287804F02DFF744B1B681A6C452101FBED
:100920000200462690FBF6F21A6493F8290028701C
:1009300004F0D6FE0523F8E06A4D287804F018FF8D
:10094000694B1B685A6C452101FB0200462690FB4F
:10095000F6F25A6493F82A00287004F0C1FE0623C8
:10096000E3E0604D287804F003FF5F4B1B689A6C4E
:10097000452101FB0200462690FBF6F29A6493F8AB
:100980002B00287004F0ACFE0723CEE0554D2878EC
:1009900004F0EEFE544B1B68DA6C452101FB0200AB
:1009A000462690FBF6F2DA6493F82C00287004F0E7
:1009B00097FE0823B9E04B4D287804F0D9FE4A4B46
:1009C0001B681A6D452101FB0200462690FBF6F2DA
:1009D0001A6593F82D00287004F082FE0923A4E024
:1009E000404D287804F0C4FE3F4B1B685A6D4521EA
:1009F00001FB0200462690FBF6F25A653B4A11784D
:100A0000092907D9987B28700021117004F068FE2D
:100A10000C238AE00131117093F82400287004F04F
:100A20005FFE002381E02F4D287804F0A1FE2E4BBD
:100A30001B681A69632101FB0200642690FBF6F231
:100A4000597B1A612A4A52F83120012182F880101C
:100A500093F89F00287004F043FE0A2365E0214DBF
:100A6000287804F085FE204B1B68D3F8A42002EB05
:100A7000C20210440A2190FBF1F2C3F8A42093F8BB
:100A80009E00287004F02CFE0B234EE0154D2878B4
:100A900004F06EFE144B1B68D3F8A02002EBC202D8
:100AA00010440A2190FBF1F2C3F8A02018792870B5
:100AB00004F016FE0E2338E00A4D287804F058FEA4
:100AC000094B1B689A68312101FB0200322690FB1A
:100AD000F6F29A60987B287004F002FE0D2324E061
:100AE000C688FF1FC488FF1FB888FF1FC588FF1F67
:100AF000C4BA0000104D287804F03AFE0F4B1B6872
:100B00005A69632101FB0200642690FBF6F2597BCF
:100B10005A610B4A52F83120012182F8001193F8F2
:100B2000B000287004F0DCFD0F23237070BD02209C
:100B3000BDE8704003F0BCBEC488FF1FB888FF1F2B
:100B4000C4BA0000FFF766BEF8B505F081FE384D67
:100B50004FF416510A2004F057F94FF4FA7005F0DB
:100B6000C3FA04F081F92F7807F00107314C002116
:100B7000802320680A4601F0BEFF2B7813F0010F96
:100B8000264609D104F070F92B78DA0705D4FFF76F
:100B9000ABFDFFF767FDF7E707BB2B78DB071DD53C
:100BA0004FF4FA7005F0A0FA234B20681F6802F09A
:100BB00028F8224903463A46214807F04FFB06F041
:100BC000CFFF0028FBD0206802F01CFB4B2005F073
:100BD0008BFA194B0A20196804F016F92F7807F0E0
:100BE000010706F0BDFF60B106F078FFFF21044663
:100BF00000223068802301F07EFFE0B204F07AF931
:100C0000EFE704F04DF970B104F05AF90021044601
:100C1000FF223068802301F06EFF094802682146F8
:100C200012689047EDE7FFF71DFDFFF75DFD9DE7BB
:100C30008491FF1FB888FF1FF891FF1F509A000092
:100C4000D091FF1F2DE9F84F804F3B6893F8C460A7
:100C500016F0100F06F0040807D0B8F1000F01D00D
:100C6000FFF772FF1B2003F023FE16F0020F784CF3
:100C7000784D0DD02268784B0AB9236001E0774A9D
:100C800013602A7802230AB9724A00E0744A13708A
:100C9000B8F1000F0DD02268724B0AB96C4A00E01F
:100CA0006E4A13602A7804230AB96A4A00E06C4A43
:100CB000137033070DD522686B4B0AB9644A00E004
:100CC000664A13602A7808230AB9624A00E0644A37
:100CD0001370F0070DD52268644B0AB95C4A00E036
:100CE0005E4A13602A7801230AB95A4A00E05C4A36
:100CF00013705F4E96F8008008F0010800218023F1
:100D000038680A4601F0F7FE2B78012B03D0544BCC
:100D10001B78012B3CD13378D9071FD42368534A61
:100D2000934208BF4D4B4C4A08BF1B68934202D107
:100D300005F0AEFA0AE04B4A934202D105F088FD75
:100D400004E0494A934201D106F058F83378DA07B3
:100D5000FCD54FF4FA7005F0C7F902E0B8F1000FC6
:100D600016D13378DB0713D52368404A934201D16B
:100D70003A4B1B68384A93424AD13E4B18684308A5
:100D800003F1376303F5D833B3FBF0F005F010FA45
:100D900096F8008008F001082068DFF8C09003682A
:100DA0009B689847A0B13868FF210022802301F09A
:100DB000A2FED9F80090D9F80030D3F800A0244B57
:100DC00018680368DB689847C1B24846D047E3E734
:100DD000D9F8000003689B689847A0B138680021E3
:100DE000FF22802301F087FED4F800A0DAF800305B
:100DF000D3F800B0194B18680368DB689847C1B294
:100E00005046D847E4E7FFF72DFCFFF76DFC75E788
:100E1000144A93420BD1174B1868430803F1376308
:100E200003F5D833B3FBF0F005F09AFCB0E70E4AB7
:100E30009342ADD10F4B1868430803F1B76303F534
:100E40005843B3FBF0F005F06DFFA1E7B888FF1F32
:100E5000D088FF1FCC88FF1F8891FF1FC888FF1F05
:100E6000CD88FF1F9891FF1FA891FF1FD091FF1FF2
:100E70008491FF1FF891FF1F38B5044608460D46C0
:100E800007F0C3FF236802465B682046294698475F
:100E900038BD38B50446FFF7EFFF0546204607F09A
:100EA000C7F9284438BDFFFF38B500250446057151
:100EB000457180F8545004491422063007F0C4FFED
:100EC0002565204638BD00BF019B000000797047B2
:100ED00090F85520044B53F83220012382F88030DB
:100EE00003711846704700BFC4BA000038B5084BFC
:100EF00090F8552053F832300124054683F800411C
:100F00000A2005F0F1F800232B71204638BD00BF00
:100F1000C4BA00004079704706307047006D7047D2
:100F200038B50446006803681B6A98472046FFF7F7
:100F3000DDFF94F856200E4B53F83230012583F82C
:100F400080500A2005F0D0F82046FFF7C1FF206846
:100F5000084B20221A6003684FF416419B6998479A
:100F600040F2EE2005F0C0F884F8545038BD00BFC0
:100F7000C4BA000084F00F4070B5044600680368EE
:100F80001B6A98472046FFF7B1FF94F856200E4B96
:100F900053F83230012283F800210A2005F0A4F82A
:100FA0002046FFF795FF2568084B20221A602B6822
:100FB0009E69074B186801F00FFE01462846B047AE
:100FC000002384F8543070BDC4BA000088F00F408C
:100FD000B888FF1F10B58EB0322201A80C4607F06A
:100FE00033FF00233A2101A88DF8353007F0EEFEDB
:100FF000014608B9207003E02046013107F0FDFEEC
:101000000EB010BD2DE9F8430025074688469146ED
:101010000D702C462E46386803689B68984748B385
:1010200038680368DB689847C0B20EB945282DD0F0
:1010300001360D28F6B203D1002308F8043009E088
:1010400009F1FF339C42F7D008F804000134E4B200
:101050000025E0E7386803689B68984738B138682E
:101060000368DB6898470A2005F03EF8F2E70120A4
:10107000BDE8F88301350A20EDB205F035F8312DD1
:10108000C9D9201C18BF0120BDE8F8833046BDE84F
:10109000F883FFFF70B5044625460679FFF740FF49
:1010A000002355F81A0B0E496371FFF7F2FE204634
:1010B00029463222FFF7A6FF38B128460949022205
:1010C00007F0ABFE08B9012300E00023637120465E
:1010D000FFF752FF16B92046FFF708FF607970BD91
:1010E000279B0000249B0000437970B50446F3B1B0
:1010F00090F854600EB9FFF713FF25460C4955F8D8
:101100001A0BFFF7C6FE322229462046FFF77AFF68
:1011100020462946FFF75EFFA01D2946142207F04E
:1011200093FE26B92046BDE87040FFF725BF70BD8D
:101130002A9B0000437970B50446EBB190F85460E7
:101140000EB9FFF7EDFE25460C4955F81A0BFFF7CF
:10115000A0FE322229462046FFF754FF20462946AA
:10116000FFF738FF284607F0E6FC206526B9204641
:10117000BDE87040FFF700BF70BD00BF339B0000AB
:1011800070B52B4D01600446286801F02EFD032840
:1011900004D1212384F85530172306E004380128B0
:1011A00037D8032384F85530182384F8563094F840
:1011B0005600012104F07AFE94F856201D4B53F896
:1011C0003230012183F8001194F8550004F06EFECE
:1011D0002046FFF77DFE2046FFF75CFF637933B3BF
:1011E0002046FFF79DFE2046FFF7A4FF2046FFF7AD
:1011F0007BFF2046FFF7C0FE2046FFF769FE24680C
:10120000286823689E6901F0E7FC01462046B04744
:101210000DE00A2003F04CFB074B063403F11402E7
:1012200053F8041B44F8041B9342F9D170BD70BD00
:10123000B888FF1FC4BA00003C9B0000F8B5437992
:1012400004460F4643B390F854600EB9FFF768FEAA
:1012500025463A461149206807F000F855F81A0B60
:101260000F49FFF709FE204629463222FFF7CAFE42
:1012700060B128460B49022207F0CFFD30B9A01D0E
:101280003946142207F0E0FD012500E0002516B9DB
:101290002046FFF771FE2B461846F8BD509B000014
:1012A000219B0000249B0000437970B504460D4645
:1012B0002BB390F854600EB9FFF732FE2A4625464C
:1012C0001049206806F0CAFF55F81A0B0E49FFF7BF
:1012D000D3FD204629463222FFF794FE48B1284626
:1012E0000A49022207F099FDD0F1010538BF002517
:1012F00000E0054616B92046FFF73EFE2B4618468D
:1013000070BD00BF129B0000219B0000249B0000C9
:10131000F8B5437904460F4623B390F854600EB9EC
:10132000FFF7FEFD25463A460F49206806F096FF76
:1013300055F81A0B0D49FFF79FFD2046294632222A
:10134000FFF760FE40B128460949022207F065FD1B
:1013500010B92765012500E0002516B92046FFF7E2
:101360000BFE2B461846F8BD5B9B0000219B00003E
:10137000249B0000F8B5437904460F4600F11A0596
:101380000BB9837615E090F854600EB9FFF7C8FDED
:1013900039462068FFF770FD07492068FFF76CFDAC
:1013A000204629463222FFF72DFE16B92046FFF7C8
:1013B000E3FD2846F8BD00BF219B0000002301216A
:1013C00010B50A460446C3600361094B4FF4BF7071
:1013D00003F0A2FA042120600122064B4FF4BF70F3
:1013E00003F09AFA42236060A360204610BD00BF5C
:1013F000689B0000799B00000A23034AB1FBF3F1CC
:10140000B2FBF1F38360704730D4050010B5044699
:10141000006807F0E1FB606807F0DEFB204610BDC6
:1014200003690268D154084A03691168426842F8A6
:1014300023105A1CB2F5BF7FA5BF6FF4BE729B1874
:1014400002610361704700BFD489FF1FC26803694E
:101450009A42CABFC2F5BF72C2EB0300D0187047F0
:1014600038B50D460446FFF7F1FF854204DB062040
:1014700003F01EFA002038BDE16823682944B1F565
:10148000BF7FA8BFA1F5BF71585C38BDC3680069B4
:101490005A1E48BF03F27D12131A58425841704732
:1014A0000023C3600361704738B50D460446FFF75B
:1014B000CDFF854204DD0820BDE8384003F0F8B9CF
:1014C000E1682944B1F5BF7FA8BFA1F5BF71E16014
:1014D00038BDFFFF38B50B4B1D6883680446ED1A15
:1014E0002046FFF7B3FF00280ADDE268636853F87F
:1014F0002230AB4204D820460121FFF7D5FFEFE7A9
:1015000038BD00BFD489FF1F014B0360704700BF87
:10151000C89B0000014B0360704700BFC89B0000E0
:1015200010B5034B0360044606F05FFE204610BD75
:10153000C89B000010B5034B0360044606F055FE3F
:10154000204610BDC89B000030B585B004AC04E94E
:101550000E00089C34B94068194905B0BDE8304018
:1015600006F07CBE9DF80430022B07D0032B1DD162
:101570001449627C406806F071FE1BE0E268637CFF
:10158000012A04D1A26840680F4912780BE0022AB0
:1015900007D1A16840680A784D780B4902EB052213
:1015A00001E04068094906F059FE03E0084809498E
:1015B00006F054FE204605B0BDE8304007F00CBBF5
:1015C000F89B0000BFA20000039C00000E9C0000DE
:1015D000D091FF1F269C0000F8B5124F124B0360FC
:1015E0000025FA26044680F87A5080F88E50416033
:1015F000426680F8485080F86050C6662A463B46EE
:101600003046012103F088F9C4F880602067012189
:1016100030462A463B4603F07FF9C4F88400204652
:10162000F8BD00BF529C0000E89B000040680149E3
:1016300006F014BE629C00002DE9F041244BDFF857
:1016400094801B888AB005A9ADF81430D8F8003012
:101650001A6800910221002400F168070191D56900
:101660008DF81D40184639460322FE23A8476D46D3
:1016700007AE45F8044B96E8070085E807002346C7
:10168000D8F800003946224603F0D0F8D8F8000018
:101690008DF819401E238DF818308DF81A4006AACF
:1016A0000368009203220192D3F81CC03946FE233E
:1016B000E047009496E8070085E807002346D8F83D
:1016C00000003946224603F0B1F80AB0BDE8F081C7
:1016D000D89B0000C088FF1F4068014906F0BEBDCE
:1016E000F19C00000A4B10B5044618680023C2188C
:1016F000013300210A2B82F88A10F8D1054B1868B3
:1017000002F05AFE60680449FFF7C3FB10BD00BF3A
:10171000B888FF1FC088FF1F689D00002DE9F341B6
:10172000674D68490446406806F098FD2868666879
:1017300001F05BFA64490246304606F08FFD2868E6
:10174000666801F058FA61490246304606F086FDA7
:101750002868666801F055FA5D490246304606F091
:101760007DFD2868D4F8048001F054FA0746286803
:1017700001F056FA0646286801F058FA33465549F2
:1017800000903A46404606F069FD2868666801F018
:1017900059FA51490246304606F060FD286801F0CA
:1017A0004BFA10B160684D4901E060684C4906F0A1
:1017B00055FD4C496068FFF75FFB2868666801F0DB
:1017C00047FA49490246304606F048FD28686768EE
:1017D00001F0D0F90646286801F0C9F932460346FF
:1017E0004249384606F03AFD2868676801F0C8F9B2
:1017F0000646286801F0D7F9324603463C49384688
:1018000006F02CFD2868666801F0D0F939490246D7
:10181000304606F023FD2868666801F0CAF9364BA9
:10182000364A3749002818BF1A46304606F016FDDA
:1018300034496068224EFFF71FFB2868D4F8048003
:1018400001F0C4F9074628682F4D01F0BCF92F4973
:1018500003463A46404606F001FD2868FFF75AFB6A
:1018600038B32B496068FFF714FB3068D4F8048064
:1018700001F0B5F90746306801F0AEF93A46034683
:101880002449404606F0EAFC28686668FFF744FBF6
:1018900021490246304606F0E1FC28686468FFF7FB
:1018A0003DFB1E490246204602B0BDE8F04106F06D
:1018B000D5BC60681A49FFF7ECFA02B0BDE8F081C8
:1018C000B888FF1FAC9D0000C99D0000D99D000095
:1018D000F49D0000099E0000259E0000489E000027
:1018E0007F9E0000B69E0000DE9E0000849F0000E8
:1018F000F79E00001D9F0000A59D0000A99D00000F
:10190000369F00004F9F0000B088FF1F769F0000A9
:10191000A49F0000D39F0000FC9F000018A00000BF
:1019200036A000002DE9F0416F4D2B680446D3F836
:10193000B40002F0B1FF6D490746606806F08EFC06
:101940002B68D4F80480986802F09CFF0A2690FB6C
:10195000F6F26749404606F081FC97FBF6F206FB7B
:10196000127364496068644F06F078FC2B68634921
:10197000D3F8AC20606892FBF6F206F06FFC2B689F
:101980005F49D3F8A42060685E4E06F067FC2B68C0
:101990005D49D3F8A020606806F060FC2B685B49C5
:1019A0001A7B6068002A0CBF3A46324606F056FCA5
:1019B0002B6857491A69606806F050FC2B68554936
:1019C0005A691B696068D21A06F048FC2B685249B4
:1019D0001A7E6068002A0CBF3A46324606F03EFC8A
:1019E0002B684E49DA69606806F038FC2B684C4970
:1019F0001A6A606806F032FC4A49606806F02EFCFC
:101A0000494B4A491A78606806F028FC484B494916
:101A10001A78606806F022FC474B48491A786068DB
:101A200006F01CFC4649606806F018FC28686668E9
:101A300001F00EF943490246304606F00FFC00263D
:101A40002B68334493F88A202AB160683E4993F8A2
:101A5000943006F003FC01360A2EF1D160683B4950
:101A600006F0FCFB012628686768821992F87F104F
:101A700006F10B0250F8228049B101F0E3F801466B
:101A8000404602F00EFF32490346384608E001F0B6
:101A9000D9F80146404602F004FF2E490346384675
:101AA0003246013606F0DAFB0B2EDCD12A4D2868CF
:101AB000FFF730FA90B129496068FFF7EAF9286822
:101AC0006468FFF703FA264B264A2749002818BF07
:101AD0001A462046BDE8F04106F0C0BB60682349C5
:101AE000FFF7D7F9BDE8F081B888FF1F6BA00000B1
:101AF0007AA0000099A00000A99D0000BAA00000F3
:101B0000E4A00000A59D000004A1000022A10000A7
:101B100045A100006CA1000096A10000B8A1000042
:101B2000D9A10000FAA10000EC91FF1F16A200004D
:101B3000D488FF1F3CA20000ED91FF1F62A20000AD
:101B400087A20000ACA20000BCA20000C5A2000059
:101B5000D4A2000004A30000B088FF1F23A300004C
:101B600064A0000067A0000052A3000036A000009F
:101B700038B5184B45680446186801F042F8164914
:101B80000246284606F06AFB6068144906F066FBC8
:101B90006068134906F062FB6068124906F05EFB5C
:101BA0006068114906F05AFB6068104906F056FB60
:101BB00060680F4906F052FB60680E4906F04EFB64
:101BC00060680D4906F04AFB60680C49BDE8384082
:101BD00006F044BBB888FF1F6EA3000098A3000066
:101BE00069A400007CA4000089A40000A2A4000055
:101BF000C4A40000F0A400000EA500002DA5000064
:101C000070B5234D46680446286800F0FAFF214964
:101C10000246304606F022FB60681F4906F01EFBB4
:101C200060681E4906F01AFB60681D4906F016FB45
:101C300060681C4906F012FB1B49606806F00EFB49
:101C40002868666800F0FBFF18490246304606F037
:101C500005FB6068164906F001FB6068154906F04F
:101C6000FDFA6068144906F0F9FA6068134906F055
:101C7000F5FA6068124906F0F1FA6068114906F059
:101C8000EDFA60681049BDE8704006F0E7BA00BFA1
:101C9000B888FF1F6EA300007BA50000BAA5000056
:101CA000CEA50000F5A500001AA6000053A600006E
:101CB0009BA60000DEA6000065A70000D0A70000DC
:101CC0000EA800004BA800007DA800004068014954
:101CD00006F0C4BAB0A800002DE9F04F03298BB07C
:101CE0000446894602D0FFF7F1FF61E0006D06F07F
:101CF00022FF8246606D06F01EFF2F4B5FFA8AFAC4
:101D000083465146186800F0ABFF10B960682B4954
:101D100004E0BBF5805F04DB6068294906F09EFAA9
:101D200046E0DFF8A480274BD8F800001B88ADF808
:101D3000143005AA036800920222002504F1680706
:101D40000192DC698DF81D5039464A465346A0473A
:101D50006C4607AE44F8045B96E8070084E8070089
:101D60002B46D8F8000039462A4602F05FFD8DF870
:101D700019B0D8F800001E234FEA2B2B8DF818302D
:101D80008DF81AB006AA03688DE804023946D3F824
:101D90001CC04A465346E047009596E8070084E891
:101DA00007002B46D8F8000039462A4602F03EFDCF
:101DB0000BB0BDE8F08F00BFB888FF1F01A900007D
:101DC0004DA90000D89B0000C088FF1F2DE9F041FD
:101DD000042988B0044602D0FFF778FF66E0006D62
:101DE00006F0A9FE0546606D06F0A5FE8046A06DD2
:101DF00006F0A1FEFF28074653DC2E4EEDB23068F8
:101E000029465FFA88F800F02BFF50B38DF8108058
:101E1000DFF8A8808DF81170D8F8000004AA00231C
:101E20008DF815300368009202220192032604F116
:101E30006807D3F81CC08DF814602B466D463946F0
:101E40003246E04745F8044B08AB13E9070085E844
:101E500007003346D8F800003946012202F0E6FCBC
:101E600024E0306800F0F4FE85421AD10A2384F899
:101E70006830032384F86A3002236367236F84F891
:101E8000695083F80080236F5F70306804F1680147
:101E900004F17C0201F07EFC6068074994F88D2013
:101EA00002E060680449082206F0D8F908B0BDE8ED
:101EB000F08100BFB888FF1FBFA20000C088FF1FCD
:101EC0002DE9F043032989B00446884602D0FFF784
:101ED000FDFE60E0006D314E06F02DFEC5B2606D76
:101EE00006F029FE2946C7B2306800F0B9FE48B3B3
:101EF000DFF8B4908DF81070D9F8000001260222A6
:101F00008DF8116004A900238DF8153003688DF851
:101F100014208DE8060004F16807D3F81CC02B4696
:101F20006D463946E04745F8044B08AB13E9070016
:101F300085E807004346D9F800003946324602F0EA
:101F400075FC28E0306800F083FE85421ED10A232C
:101F500084F86830022384F86A306367236F84F85A
:101F600069501F70236F01225A70306804F16801B4
:101F700004F17C0201F070F9D4F8843060681A78BA
:101F8000074994F88D3006F069F904E06068054966
:101F9000082206F063F909B0BDE8F083B888FF1F96
:101FA000039C0000BFA20000C088FF1F2DE9F04184
:101FB000042988B0044602D0FFF788FE66E0006D71
:101FC000344F06F0B8FDC5B2606D06F0B4FD5FFA9F
:101FD00080F8A06D06F0AFFD29460646386800F08F
:101FE0003FFE60B38DF81080DFF8B0808DF811608F
:101FF000D8F8000036128DF8126004AA03260023D8
:102000008DF8153003688DF814608DE8440004F1F4
:102010006807D3F81CC02B466D4639463246E04768
:1020200045F8044B08AB13E9070085E80700334681
:10203000D8F800003946012202F0F8FB26E03868A3
:1020400000F006FE85421CD10A2384F86830032381
:1020500084F86A306367236F84F8695083F80080DE
:10206000236F5E70236F36129E70386804F168012A
:1020700004F17C0201F08EFB6068074994F88D2022
:1020800002E060680449082206F0E8F808B0BDE8FC
:10209000F08100BFB888FF1FBFA20000C088FF1FEB
:1020A0002DE9F041032988B004460E4602D0FFF71F
:1020B0000DFE63E0006D334F06F03DFDC5B2606D6F
:1020C00006F039FD29465FFA80F8386800F0C8FD4F
:1020D00040B38DF81080DFF8B8800222D8F80000F5
:1020E0008DF8112004A900238DF8153003688DF8B0
:1020F00014208DE8060004F16807D3F81CC02B46B5
:102100006D463946E04745F8044B08AB13E9070034
:1021100085E807003346D8F800003946012202F06E
:1021200085FB2BE0386800F093FD854221D1226FBA
:1021300084F869500A2384F86830022384F86A30EE
:10214000666782F80080226F5370386804F1680176
:1021500004F17C0201F080F8D4F8843060681A78C9
:102160005B78094902EB032294F88D3006F076F88B
:1021700004E060680549082206F070F808B0BDE880
:10218000F08100BFB888FF1F039C0000BFA20000C1
:10219000C088FF1F022938B5044604D02046BDE898
:1021A0003840FFF793BD056D0E49284606F01BFE2B
:1021B00040B90D4B186801F025F860680B49FEF72F
:1021C00068FE38BD28460A4906F00DFE0028E5D114
:1021D000054C206800F0F6FF2068BDE8384001F0AB
:1021E0001FB800BFB5A90000B888FF1FB9A900003B
:1021F000BEA90000022910B5044603D0BDE8104076
:10220000FFF764BD006D06F096FC094BC1B218687B
:1022100001F00EF830B96068226D0649BDE8104043
:1022200006F01CB860680449FEF733FE10BD00BF1D
:10223000B888FF1FC2A9000008AA0000032970B5D2
:1022400004461AD1056D6B49284606F0CCFDC8B985
:10225000656D6949284606F0C6FD18B9674B01212E
:10226000186807E06649284606F0BDFD014620B91A
:10227000624B186800F0A0FC71E02046BDE8704099
:10228000FFF724BD28465F4906F0ADFDA8B9656D8E
:102290005949284606F0A7FD18B9584B012118687E
:1022A00008E05749284606F09EFD01460028E4D183
:1022B000524B186800F0F2FC51E02846524906F0F3
:1022C00092FD48B94D4B606D1D6806F034FCC1B2FB
:1022D000284600F07EFC42E028464C4906F083FD8B
:1022E000002841D1606D06F02AFCCF28054602DDAA
:1022F0006068474935E0474B013093FBF0F006F04A
:10230000B5F9454906F0BAFA0021064606F0B4FBD5
:1023100028B130464FF07C5106F0F4F804E0304626
:102320004FF07C5106F0ECF806F0BAFB3B4A03464E
:102330004FF4165110685943FEF7B6FF10B16068AC
:10234000374901E06068374905F088FF2B4BE9B257
:10235000186800F047FC60683349FEF79AFD606832
:102360003249FEF796FD70BD2846314906F03BFD27
:1023700070B92A4B616D1868FEF760FF10B1606894
:102380002C4901E060682C49BDE8704005F066BF4B
:1023900028462A4906F027FDC0B9606D06F0CBFB40
:1023A00042F20F739842014602DD60682449EBE770
:1023B0001A4D2868FEF7ACFF0028E3D0286864684F
:1023C000FEF7ACFD1F49024620460FE028461E4995
:1023D00006F009FD00287FF450AF104B616D1868BE
:1023E0006568FEF7C7FF194902462846BDE87040F8
:1023F00005F034BF0EAA00001AAA0000B888FF1F1B
:102400001EAA000021AA000031AA000039AA00007B
:1024100040AA000080841E0000001646B088FF1FFE
:102420008CAA0000ABAA0000CAAA0000B9A900004B
:10243000EEAA0000F5AA0000FDAA000003AB000010
:102440000AAB000058AB00008FAB000099AB000056
:10245000022970B504460D4608D1006D3C4906F0CE
:10246000C2FC002849D102F07DFB6BE0032944D176
:10247000056D3849284606F0B6FC48B9364B606D04
:102480001D6806F058FB0146284600F0B1FB59E0F4
:102490002846324906F0A7FC48B92F4B606D1D68ED
:1024A00006F049FB0146284600F0A8FB4AE0284612
:1024B0002B4906F098FC48B9274B606D1D6806F063
:1024C0003AFB0146284600F0C0FB3BE02846254980
:1024D00006F089FCB0B9656D2349284606F083FCF7
:1024E00008B9282005E02846204906F07CFC48B9B8
:1024F0001E20012102F01CFB24E0206D1C4906F087
:1025000072FC20B12046BDE87040FFF7DFBB052D0F
:10251000F8D1114D606D2E6806F00DFBC1B230464A
:1025200000F07BFBA06D2E6806F005FBC1B23046C3
:1025300000F079FBE06D2D6806F0FDFAC1B2284687
:1025400000F077FB60680B49FEF7A3FC70BD00BF8D
:10255000A4AB0000ABAB0000B888FF1FB6AB000017
:10256000C4AB0000D4AB0000DFAB0000E4AB000064
:10257000EAAB0000B9A90000F8B501230B7090F890
:1025800048303F2B84BF03F1FF3380F8483090F888
:10259000482002440023137204460E46012294F898
:1025A0004800D9B288420CD92144097A202905D1A2
:1025B0002AB9327801323270012200E00022013360
:1025C000EDE73378052BA8BF0523337004F1080528
:1025D000002384F8603094F860703378BB421CD9D3
:1025E0002846202194F8482006F0FEFA30B904EB82
:1025F00087030137DD6484F86070ECE7A84201D1FD
:102600000135E8E704EB87070023FD64054605F87C
:10261000013B94F860300133DBE7E46C434920462A
:1026200006F0E1FB002860D02046414906F0DBFBC4
:1026300000285CD020463F4906F0D5FB002858D042
:1026400020463D4906F0CFFB002854D020463B49A8
:1026500006F0C9FB002850D02046394906F0C3FBDC
:1026600000284CD02046374906F0BDFB002848D052
:102670002046354906F0B7FB002844D020463349B0
:1026800006F0B1FB002840D02046314906F0ABFBF4
:1026900000283CD020462F4906F0A5FB002838D062
:1026A00020462D4906F09FFB002834D020462B49B8
:1026B00006F099FB002830D02046294906F093FB0C
:1026C00000282CD02046274906F08DFB48B3204631
:1026D000254906F088FB30B32046244906F083FBE9
:1026E000002814BF01201120F8BD0220F8BD0320EE
:1026F000F8BD0420F8BD0520F8BD0620F8BD072070
:10270000F8BD0820F8BD0920F8BD0A20F8BD0B204F
:10271000F8BD0C20F8BD0D20F8BD1220F8BD0E202C
:10272000F8BD0F20F8BD1020F8BD00BFEDAB0000D4
:10273000F2AB0000F6AB0000FDAB000003AC000004
:1027400015AC00000BAC000011AC00001AAC00008E
:1027500021AC000011AD0000BDAB000029AC0000B1
:1027600034AC000038AC00003CAC000040AC0000D1
:1027700013B50446606803689B689847002800F01A
:102780008B8060680368DB689847C0B20D28F1D081
:102790000A2894F8483001D1012B01D83F2B75D17C
:1027A00020460DF10701FFF7E7FE122867D8DFE8A2
:1027B00000F0730A0E12161A1E22262A30363C42E8
:1027C0004E545A6048002046FFF780FA5AE02046EF
:1027D000FFF716FA56E02046FFF7CAF952E0204606
:1027E000FFF7A0F84EE02046FEF798FF4AE02046AB
:1027F000FEF778FF46E02046FEF71EFF42E0204647
:10280000FEF76AFF3EE020469DF80710FEF70EFF38
:1028100038E020469DF80710FFF75EFA32E02046C8
:102820009DF80710FFF7B6FC2CE020469DF8071036
:10283000FFF70EFE26E020469DF80710FFF7FEFC8E
:1028400020E020469DF80710FFF7D4FC1AE0204650
:102850009DF80710FFF7BAFA14E020469DF807101C
:10286000FFF7A4FB0EE020469DF80710FFF728FBBA
:1028700008E020469DF80710FFF712FC02E00D204B
:1028800002F016F8002384F8483005E05A1C23446F
:1028900084F8482018726DE702B010BD10B50446E8
:1028A00000F026F8204610BDF0B589B06B46002434
:1028B0008DF8154043F8044B08AF06460D4617E95E
:1028C000070083E80700304629462246234600F0E9
:1028D00080F809B0F0BD08B500F0BDF8043008BDBF
:1028E00000F0F4B800F0FEB800F0F3B800F0FCB867
:1028F000F8B504460D4616460846002228212A4B04
:1029000002F00AF8294B2061012106FB05F00022A4
:1029100002F002F800236061DAB2AA4208D222690A
:10292000282101FB03220133D06096603044F3E795
:102930000C2101221E4B284601F0EEFF0C266FF001
:102940000B01034600F10C0216FB0511606006FB4B
:10295000053682605A1820691860183E5A60566021
:10296000282606FB0506283E5E5093600122691E5C
:102970008A4213DA0C2112FB01F601FB023C9F197B
:1029800011FB021119444CF8087CB96002EB82017A
:1029900000EBC10101329951D2B2E8E7A360E360D4
:1029A000002323702046F8BD44AC00005DAC00005D
:1029B00081AC000010B50446406906F00DF92069AD
:1029C00006F00AF9606806F007F900232370204634
:1029D00010BD2DE9F8439046027899460446836875
:1029E00012B91D46E36009E0C568AA689A4205D19C
:1029F000192001F05DFF0020BDE8F8832E68E36830
:102A0000B2689B68F068E3600F46331D01F1140E55
:102A100057F804CB43F804CB7745F9D1CB68B260C3
:102A2000F0609A42A8BF1A463261896802F02CFC15
:102A30002968089A81F825902B6881F8248043F84A
:102A4000182B09AA07CA83E80700237801332370EB
:102A50000120BDE8F88310B5047814B183681868C4
:102A600010BD152001F024FF204610BD38B50378B5
:102A70008B4204460D4604DC1720BDE8384001F0C7
:102A800017BF19B983689B6883601BE0013B9942BB
:102A900003D1C3685B68C36014E0182001F008FF2D
:102AA000A368013D15F0FF059B68FAD15A68996843
:102AB000916099684A60E2689168996091685A608B
:102AC0004B6093602378013B237038BD0021FFF7F2
:102AD000CDBF10B5044623781BB12046FFF7F6FFA3
:102AE000F9E710BD00787047C36880689A68131AC8
:102AF00058425841704710B580F8CA3090F8C83035
:102B000080F8C910044680F8CB2090F8C50093B136
:102B1000C943C9B2013103F0E5F994F8CB1094F838
:102B2000C600C943C9B2013103F0DCF994F8CA10F8
:102B3000C943C9B20BE0013103F0D4F994F8CB10CA
:102B400094F8C600013103F0CDF994F8CA1094F856
:102B5000C7000131BDE8104003F0C4B990F8C900C6
:102B6000704790F8CB00704790F8CA007047D0F8D3
:102B7000D000704790F8CC0070470B2001F0A4BF44
:102B800090F8D400704738B50546084685F8D4104B
:102B90000C4601F075FE2146C5F8D8000C20BDE8B2
:102BA000384001F091BFD0F8D800704790F8DC00B1
:102BB000704790F8DE0070470A461720012102B1E5
:102BC0000A4601F031BFD0F8E000704790F8DF000E
:102BD00070470F2001F078BFD0F8E800704790F8F8
:102BE000E4007047102001F06FBFD0F8EC00704790
:102BF000002001F083BFD0F8F0007047022001F000
:102C00007DBF90F8F900704780F8F9100A201A216A
:102C100001F05ABF90F8FA007047042001F054BF49
:102C200090F8FB007047052001F04EBF90F8FC00C3
:102C30007047062001F048BF90F8F8007047D0F8C0
:102C4000F4007047D0F8000170471A2001F056BF19
:102C500090F8DD00704780F8DD100E2001F034BFE1
:102C600059B10023C21892F88A208A4203D0013356
:102C70000A2BF7D101E0012070470020704702467F
:102C800049B100231846D31893F88A308B4204D0F8
:102C9000431C0A2BF6D14FF0FF3070470A4617202D
:102CA000002101F0C1BE90F8FD1010B50446B1B985
:102CB000D0F8EC3090F8A900032B02D103F0F6F81D
:102CC00007E0012103F0F2F894F8A900012103F0D4
:102CD000CDF8322003F008FA012384F8FD3010BD4E
:102CE0002DE9F04104460A2001F092FE1A2884F8EA
:102CF000F90003D020461A21FFF786FF002001F0DB
:102D00008DFEC4F8EC00022001F088FEC4F8F0004B
:102D10000D2001F07DFE84F8DC000C2001F078FE2F
:102D200084F8D40001F0ACFDC4F8D8000B2001F009
:102D30006FFE84F8CC0001F089FD0121C4F8D000B9
:102D4000172001F053FE003018BF012084F8DE0088
:102D50000E2001F05DFE84F8DD000F2001F058FE2A
:102D600084F8DF0001F072FDC4F8E000102001F0EB
:102D70004FFE84F8E40001F069FDC4F8E800042087
:102D800001F046FE84F8FA00052001F041FE84F8C7
:102D9000FB00062001F03CFE002184F8FC0084F8D2
:102DA000C410172001F022FE003018BF012084F863
:102DB000F80010B140F6FF7301E040F2FF33C4F8B1
:102DC000F430D4F8F03003F001022273C3F3400270
:102DD00022765A0701D5322304E01B074CBF4A2351
:102DE0004FF0FF330025C4F8AC3084F8FD501A20B2
:102DF00001F014FED4F8F030C4F8000113F0160FFF
:102E00000CBF0023012384F8C8304FF44873C4F882
:102E1000B8304FF49663C4F8BC30012140F2DC5363
:102E2000C4F8C0300A200A46D64B01F075FDD4F82C
:102E3000EC702060032F79D102234FF0040884F84E
:102E4000A8304046012184F8C58003F02FF8052002
:102E500084F8C600012103F029F8062084F8C70091
:102E6000012103F023F82A46772320463321FFF778
:102E700042FE12200121607303F018F82520A07390
:102E800002F0BEFB19236061637620610F230B20E3
:102E9000A376012184F8AA00242603F007F81D2058
:102EA00084F8B060207102F0ABFBA06094F8B00031
:102EB00002F0A6FB1A2384F824301C2384F8253062
:102EC000152384F82630102384F827301F2384F834
:102ED000A930C4F8B4002946092084F8286084F891
:102EE000296084F82A6084F82B6084F82C6084F8C8
:102EF0002D6084F89E6084F89F6002F0D7FF202048
:102F0000294602F0D3FF3846294602F0CFFF0C20B5
:102F1000012102F0CBFF9C4B80221A60132001217B
:102F200002F0C4FF994BC3F800800AE1042F70D16E
:102F3000022384F8A830384684F8C570012102F0D5
:102F4000B5FF052084F8C600012102F0AFFF06207E
:102F500084F8C700012102F0A9FFFF222B4620467A
:102F60002946FFF7C8FD1E206073012102F09EFF75
:102F70001D20A07302F044FB192360616376206179
:102F8000212320200121A37684F8AA0002F08EFFDD
:102F90001F230F2084F8B030207102F031FBA060B5
:102FA00094F8B00002F02CFB1C2384F824301B237F
:102FB00084F82530242384F82630252384F827300C
:102FC000112384F82830132384F82930142384F83B
:102FD0002A30152384F82B30172384F82C3016233D
:102FE00084F82D30122384F89E301A23C4F8B400DC
:102FF00084F89F301020012102F058FF294610204C
:1030000002F034FF0E2084F8A900012102F04EFFE7
:1030100097E0052F40F091800223152084F8A83016
:1030200084F8C500012102F041FF384684F8C670DB
:10303000012102F03BFF062084F8C700012102F0C5
:1030400035FFFF222B4620462946FFF754FD14206A
:103050006073012102F02AFF1020A07302F0D0FA61
:103060001923606163762061212320200121A3764A
:1030700084F8AA0002F01AFF1F230F2084F8B03052
:10308000207102F0BDFAA06094F8B00002F0B8FA26
:103090001C2384F824301B2384F82530242384F84F
:1030A0002630252384F82730112384F82830132371
:1030B00084F82930232384F82A30222384F82B3003
:1030C000172384F82C30162384F82D301223C4F8EB
:1030D000B40084F89E300E201A2384F89F3084F8C0
:1030E000A900012102F0E2FE0920012102F0DEFE2A
:1030F0002946092002F0BAFE0B20012102F0D6FE7B
:1031000029460B2002F0B2FE0C20012102F0CEFE77
:1031100029460C2002F0AAFE1D20012102F0C6FE65
:1031200029461D2002F0A2FE1E20012102F0BEFE53
:103130001E20294602F09AFE03E0FE23C4F8EC307C
:103140003CE02046FFF7AFFD207902F059FA237EDC
:10315000A06043B1607E04F039F8E061A07E04F025
:1031600035F8206201E0E3612362237B83B1607B59
:10317000012102F09BFEA07B02F042FA206123694C
:1031800007E000BF03AD000088F00F4048F00F409B
:103190002361636104F10A062546002385F88A301D
:1031A000A36595F8240085F880302F1B02F028FADB
:1031B0000C370135B54244F82700EED12046BDE872
:1031C000F08100BF10B5D0F8EC30032B044690F826
:1031D000A9000ED1012102F069FE94F8A920084B44
:1031E00053F83230012283F880200A2002F07CFF5D
:1031F00002E0002102F03AFE002384F8FD3010BD09
:10320000C4BA000010B50446FFF7DCFF4FF4967017
:1032100002F06AFF2046BDE81040FFF744BDFFFF03
:10322000014B024A1A6070470CED00E00400FA05F9
:1032300011F0E0020ED10B4633B113F0010F1CBFA9
:103240000132D2B25B08F7E7022A03D180F8C4103A
:1032500001207047002070472DE9F74F8B68144616
:1032600093F800905A78636809F1FF3A9A42B8BF20
:1032700013469A444FF00008DBB2E36084F81180F3
:103280000546FFF7DFFC5FFA8AFA074609EB0803F9
:10329000DBB2534500F270825FFA88F6B82B00F279
:1032A0006582DFE813F0B9004301BC00C200C8002A
:1032B000630263026302CE00D4006302630263020E
:1032C000630263026302DE00630263026302E400DE
:1032D00063026302630263026302630263026302C6
:1032E00063026302630263026302630263026302B6
:1032F00063026302630263026302EA00F100630295
:103300006302630263026302630263026302630295
:103310006302630263026302630263026302FA00F0
:103320006302000106010C011201180163021E0173
:103330002E0163023501430163023B0163023D013B
:1033400043016302460163024901510163024F01D7
:1033500063025101700154015B0162016901630262
:1033600075017801830163028E01910198019F012B
:10337000A6016302AD01B501BD01CA016302DA0114
:10338000DE01E201E601EA01EE01F201F601FA01D5
:10339000FE01020206020A020E02120216021A02BE
:1033A0001E022202290263023302360239023C0263
:1033B0003F024202450248024B024E026302630290
:1033C00063026302630263026302630263026302D5
:1033D00063026302630263026302630263026302C5
:1033E00063026302630263026302630263026302B5
:1033F00063026302630263026302630263026302A5
:1034000063025102630253026302560263025902CD
:1034100063025C0263025F02A3689522A8E128466A
:10342000D4F808B0FFF7EDFB6DE12846D4F808B0FA
:10343000FFF70EFC67E12846D4F808B0FFF79AFBC7
:1034400061E12846FFF7F8FBA368FF2290E12846D8
:10345000D4F808B0FFF7F0FB00280CBF03230F23BC
:10346000F8E02846D4F808B0FFF7A0FB4BE1284667
:10347000D4F808B0FFF7E0FB45E1D5F8B400D4F884
:1034800008B001F009FA3EE1A868D4F808B001F0EC
:10349000F9F90A2390FBF3F035E12846D4F808B097
:1034A000FFF7A3FB2FE12846D4F808B0FFF7A3FBF2
:1034B00029E12846D4F808B0FFF79DFB22E1284611
:1034C000D4F808B0FFF7A6FB1DE12846D4F808B0F1
:1034D000FFF7A6FB17E12846D4F808B0FFF7A6FBD4
:1034E00011E1A26801922846FFF73BFB834628467C
:1034F000FFF734FB2BF00F03019A03EB20109055DC
:1035000037E12846D4F808B0FFF72EFB0011FAE0A7
:103510002846D4F808B0FFF74CFBF4E0984B09E0DC
:103520002846D4F808B0FFF751FBECE0A36801226D
:103530001EE1944B1A7817E12846D4F808B0FFF73B
:103540004EFBE0E0904BF5E7A368032210E18F4BC0
:10355000D4F808B01868FDF7DDFCD4E08B4BD4F844
:1035600008B01868FDF7B2FCCDE0884BD4F808B07D
:103570001868FDF7D3FCC6E0844BD4F808B018688F
:10358000FDF7CCFCBEE0824B1B6893F8C420EBE057
:10359000A3682A7BECE02846D4F808B0FFF74CFB80
:1035A0006A692B69D31A23EAE37340E02846D4F80A
:1035B00008B0FFF741FB6A692B69D31A23EAE3736A
:1035C00042E0A3682A7ED3E02846D4F808B0FFF78B
:1035D00033FBEB692BE02846D4F808B0FFF72CFB4F
:1035E000EB6931E02846D4F808B0FFF725FB2B6AD9
:1035F0001DE02846D4F808B0FFF71EFB2B6A23E035
:103600002846D4F808B0FFF717FBD5F8A4300EE031
:103610002846D4F808B0FFF70FFBD5F8A43013E024
:103620002846D4F808B0FFF707FBD5F8A03008B15A
:10363000DBB20FE0C3F387030CE02846D4F808B0F0
:10364000FFF7FAFAD5F8A03010B1C3F3072301E071
:10365000C3F387230BF806308BE0D4F808B0286B4F
:1036600046E0D4F808B0286B49E0D4F808B0686B9D
:103670003EE0D4F808B0686B41E0D4F808B0A86B1D
:1036800036E0D4F808B0A86B39E0D4F808B0E86B9D
:103690002EE0D4F808B0E86B31E0D4F808B0286C1C
:1036A00026E0D4F808B0286C29E0D4F808B0686C9B
:1036B0001EE0D4F808B0686C21E0D4F808B0A86C1B
:1036C00016E0D4F808B0A86C19E0D4F808B0E86C9B
:1036D0000EE0D4F808B0E86C11E0D4F808B0286D1A
:1036E00006E0D4F808B0286D09E0D4F808B0686D99
:1036F000394601F0D6F806E0D4F808B0686D3946CE
:1037000001F0CFF800120BF8060032E095F88A209D
:103710002AE095F88B2027E095F88C2024E095F896
:103720008D2021E095F88E201EE095F88F201BE07B
:1037300095F8902018E095F8912015E095F89220E2
:1037400012E095F893200FE02B68F3E62B685A7887
:103750000AE02B689A7807E02B68DA7804E02B6897
:103760001A7901E02B685A79A36801E0A368002266
:103770009A5508F1010889E503B0BDE8F08F00BF54
:10378000EC91FF1FD488FF1FED91FF1FB088FF1F32
:10379000B888FF1F2DE9F74F8B6893F800A0CB681E
:1037A0000AEB030B0027ABF1020B054689461646D0
:1037B0005FFA8BFBD7605774B846FAB202EB0A0384
:1037C000DBB201325B45D2B200F2FA80D9F80810C0
:1037D000822B8C5C00F0CD803ED8442B00F08B8097
:1037E00015D8052B00F0EA8009D8032B65D0042BEF
:1037F00040F0E08028462146FFF7BFF9DEE0142BB9
:103800006DD0432B73D0102B40F0D48060E05A2B46
:1038100000F08B8018D8572B00F09B80592B7BD061
:10382000452B40F0C7802846FFF798F90146284607
:103830000191FFF796F904F00F0404EB041302461C
:1038400001992846DBB264E0802B00F0898000F209
:103850008D805B2B6BD0ADE0892B00F0998015D863
:10386000852B00F08C8009D8832B00F08580842B79
:1038700008BF85F88D4000F0A1809BE0872B00F009
:10388000818000F2828085F88F4097E0B22B00F0B3
:10389000888009D8AE2B7ED0B02B7FD08A2B40F009
:1038A000898085F8934089E0B62B7DD0B82B7ED0F7
:1038B000B42B7FD12B68DC7080E028462146FFF7CF
:1038C000CFF9002876D128462146FFF7C4F975E0E4
:1038D000022C6FD828462146FFF755F96EE028469E
:1038E0000CB9214600E00021FFF7D8F966E0284630
:1038F000FFF788FC62E02846FFF736F904F00F0175
:10390000241101EB011104EB04120346C9B228464D
:10391000D2B2FFF7F0F851E02B4B186814B9FDF75D
:10392000E5FA4BE0FDF7D4FA48E0A04646E008EBA4
:10393000042142F20F73994204DC234B1868FDF70F
:10394000E7FC03E0737C43F0080373744FF0000856
:1039500034E01E4B21461868FFF76AFC70B329E07B
:1039600064B31B4B186800F027FD27E085F88A40F8
:1039700024E085F88B4021E085F88C401EE085F836
:103980008E401BE085F8904018E085F8914015E0E6
:1039900085F8924012E02B681C700FE02B685C7079
:1039A0000CE02B689C7009E02B681C7106E02B680A
:1039B0005C7103E0737C43F0080373740137FCE629
:1039C00003B0BDE8F08F00BFB088FF1FB888FF1FAD
:1039D000C088FF1F38B5856A084B036004462DB1C7
:1039E0002846FEF7E7FF284604F0FFFB201DFDF701
:1039F0000DFD034B2360204638BD00BF20AD000005
:103A0000C89B000010B50446FFF7E4FF204604F011
:103A1000ECFB204610BDFFFF10B5002241600446BC
:103A2000034B0846012100F077FFA06010BD00BFE6
:103A3000529C00002DE9F04106461B4B46F8043B22
:103A400004469046002530460F46FDF7B7FC304649
:103A5000414684F82C5084F8425084F8565084F83B
:103A60006A502577FDF7C8FC04F13000A761FA2100
:103A7000FFF7D2FF04F14400FA21FFF7CDFF04F174
:103A80005800FA21FFF7C8FF182004F0ACFB0F2103
:103A900002220646FEF702FF0123A66284F82C509C
:103AA00023772046BDE8F08120AD000038B50446FC
:103AB000806903689B689847E8B1251D2846FDF793
:103AC00009FDA06903689B68984718B12846FDF76F
:103AD000DDFC38B194F82C301BB1074B1B686362D6
:103AE00038BD38BDA0690368DB689847C1B2284675
:103AF000FDF796FCE5E738BDD489FF1F82B030B5ED
:103B000085B00C4608A981E80C006B4643F8040B0D
:103B100007C983E80700064B9DF82C20186821464A
:103B2000032300F083FE05B0BDE8304002B07047CB
:103B3000C088FF1F10B586B000240193059B009339
:103B40008DF80D408DF80C2003AB0CCBFFF7D6FFA2
:103B500006B010BD10B50446806AFEF7C5FE00230E
:103B600084F82C3010BD38B54C78CB6802341C4436
:103B70000B780A2B0D46E4B201D18B7802E0142BAE
:103B800003D14B7C1C44E4B202E00E2000F090FE16
:103B9000E96800238B4205DAAA68D25C1444E4B2D7
:103BA0000133F7E7E043C0B238BD832906D003D81C
:103BB0000139022904D801E0922901D1012070477E
:103BC0000020704738B50446806903680D461B68BD
:103BD000FF219847A0690368FF211B689847A069E7
:103BE000697803681B689847A069E968036802312F
:103BF0001B68C9B29847A069697C03681B6898472D
:103C0000A069A9680368EA685B689847A069297C8D
:103C100003681B68984738BD70B5142380F844309A
:103C20008B780022013B04460D4680F85520052B79
:103C300026D8DFE803F003081325251E6B7880F8EB
:103C4000453002651CE06B7880F845301F4B2946F3
:103C5000186804F14402FFF7FFFA11E06B7880F86E
:103C600045301A4B2946186804F14402FFF792FDCB
:103C700006E0164E3068FFF7A5FA3068FFF7D0FA75
:103C800094F84530FE2B1FD0AB7CEBB90F4E30685B
:103C9000FEF78CFF022809D03068FEF787FF012865
:103CA000AB7801D1022B01D0012B0DD104F14405D9
:103CB00029462046FFF757FF84F85400294620463E
:103CC000BDE87040FFF77EBF70BD00BFB888FF1F22
:103CD0002DE9F04F8B6885B01A7893F801B0039204
:103CE00007460D460224EB689C4246DADFF89480D2
:103CF000AB68D8F800001E5DFEF7AAFF86420BF104
:103D0000010A05D0D8F800003146FEF7A9FF00B33C
:103D1000AB68039A1A551A4B1868AB6802682344BB
:103D200000935FFA8AF3019307F15809D2F81CC097
:103D3000494603223346E047D8F80000FEF788FFE3
:103D4000864209D1012387F86A3038464946FFF791
:103D500063FF5444E4B2C6E70A4B31461868FEF7E5
:103D60007FFF30B13846494602220123FFF7E2FEC9
:103D7000EFE7122000F09CFDEBE705B0BDE8F08F07
:103D8000C088FF1FB888FF1FF8B50446A06AFEF779
:103D9000A9FD002804DC2046BDE8F840FFF7DABEA4
:103DA000A06A174FFEF797FD457806463868FEF77C
:103DB0004FFF85423146204602D1FFF72DFF03E039
:103DC00003220123FFF7B6FEA06AFEF789FD0D4B23
:103DD00038681B686362FEF73BFF85420FD1A06A1B
:103DE000FEF780FD002806DDA06AFEF774FDC37CA7
:103DF000AB42CBD0F8BD94F82130AB42CBD0F8BD6C
:103E0000B888FF1FD489FF1F38B5012380F82C30F4
:103E1000084B90F820501B6843620446806AFEF706
:103E20005AFD4378AB4204D12046BDE83840FFF745
:103E3000ABBF38BDD489FF1F2DE9F0438B689B7859
:103E400080F820308A68CB68134485B013F8023CB0
:103E500080F8213005460C4601264FF0FF08E36844
:103E60009E423ADA771CDFF88490A368D9F8000004
:103E7000D95DFEF7F5FE38B9D9F80000FEF7E8FE87
:103E8000A368DB5D834222D1A86AFEF72FFD10B143
:103E90001A2000F00DFDA3689A1905F158099278CF
:103EA0008DF80C209A5D8DF80D200F4ADB5D1068AF
:103EB00003AA0168009202220192D1F81CC049466F
:103EC000E04785F86B80A86A4946FEF7EDFCA368D9
:103ED000033613F80780F6B2C1E72846FFF794FFD0
:103EE00005B0BDE8F08300BFC088FF1FB888FF1F82
:103EF000037F2DE9F0470446002B00F0DF8090F8A7
:103F00002C302BB16E4B1A68436AD31A642B19D824
:103F10002046FFF7CBFD251D2846FDF797FA05281B
:103F20000EDD28460021FDF79BFAFF2840F0C180F6
:103F300028460121FDF794FAFF2840F0BA8004E0FA
:103F4000BDE8F087FFF706FEE2E702212846FDF70D
:103F500087FA002384F8310084F842302846032190
:103F6000FDF77EFA0128074607DD2846FDF76EFAC1
:103F7000FB1C834203DBBDE8F087BDE8F08794F8C3
:103F80002C304BB1142384F8303028460421FDF73F
:103F900067FA84F8410008E00A2384F830302846A4
:103FA0000421FDF75DFA84F83200626BBB1E934278
:103FB000A8BF134603F10508E3635FFA88F80526F6
:103FC000F3B243450BD231462846D4F83890FDF77A
:103FD00047FAA6F1050A013609F80A00F0E741465A
:103FE0002846FDF73DFA04F1300684F840003146DA
:103FF0002046FFF7B8FD94F84030834259D194F839
:104000002C3083B1A06AFEF76DFC002845DDA06A64
:10401000FEF761FC94F83130C27C9A423DD12046D3
:10402000FFF7B2FE42E0204694F83210FFF7BDFDE4
:1040300000283BD0DFF88C8094F83190D8F800004D
:10404000FEF706FE814523D0D8F8000094F8311021
:10405000FEF706FE034630B10122204631461346E4
:10406000FFF768FD22E094F83120FE2A1ED194F873
:104070003220832A2046314602D1FFF729FE15E07F
:10408000922A02D1FFF7D8FE10E00222FFF752FD7C
:1040900020463146FFF7C0FD08E094F8212094F84F
:1040A00031309A4202D12046FFF754FD2846391D8F
:1040B00001E028460121FDF7F7F92CE7BDE8F0877C
:1040C000D489FF1FB888FF1F30B585B004AD05E95E
:1040D0000E00089D9DF804300446002D34D0012BBD
:1040E00005D1294605B0BDE83040FFF76BBD032B75
:1040F00022D190F82C30A3B12946FFF763FD134B72
:10410000A06A1B686362FEF7EDFB002809DDA06A68
:10411000FEF7E1FB6B78C27C9A4202D12046FFF7A2
:1041200033FE6A7894F821309A420DD1204605B0CA
:10413000BDE83040FFF70EBD022B05D0132005B0BF
:10414000BDE8304000F0B4BB05B030BDD489FF1FDE
:1041500038B5056D074B036004462DB12846FDF7C1
:1041600055F9284604F041F8204600F02FFB204680
:1041700038BD00BF38AD000010B50446FFF7E8FFBA
:10418000204604F032F8204610BD2DE9F04186B0FB
:1041900004688DF814209846022205AB8E4600F183
:1041A0003C07009301920126734639468DF815604D
:1041B000E4690546A0476C460CAB44F8048B93E8D1
:1041C0000700032384E8070028463946324600F0FA
:1041D0002DFB06B0BDE8F081F0B587B000F13C05DD
:1041E0008DF8153005AB8DF814200268009302237A
:1041F00001930F46D66929463B4603220446B04741
:104200006B460C9A43F8042B0DAA07CA83E80700F3
:10421000204629469DF840209DF8443000F006FBDA
:1042200007B0F0BDF0B587B004688DF814201F46C4
:10423000022205AB8E4600F13C06009301927346C4
:104240008DF815203146E4690546A0476C460CAB55
:1042500044F8047B93E80700032384E8070028461A
:104260003146012200F0E2FA07B0F0BDF0B587B0A8
:1042700006688DF815301B128DF814208DF8163055
:10428000032205AB00F13C05009301920F463B462B
:104290002946F6690446B0476B460C9A43F8042B4E
:1042A0000DAA07CA83E80700204629469DF840204A
:1042B0009DF8443000F0BAFA07B0F0BD2DE9F041A6
:1042C00088B005AC84E80E009DF814200E9B9DF884
:1042D00016509DF81780012A064632D14BB1092DA0
:1042E00035D81C495B7809686A1C0D4485F88A300A
:1042F000D5B2B8F1FC0F2AD8092D28D8326800238E
:1043000008F10108009301935FFA88F806F13C0771
:10431000D2F81CC03046394643460122E0476B467E
:104320008DF816508DF8178043F8046B94E8070059
:1043300083E80700304639460122032300F076FA6D
:1043400005E0042008B0BDE8F04100F0B1BA08B0C3
:10435000BDE8F081B888FF1FF8B5044617460E4641
:10436000002500F051FA134B2360666584F826504F
:1043700084F83A5084F84E50142003F034FF064677
:10438000FDF71CF8304639462665FDF735F804F18F
:104390001400FA21FFF740FB04F12800FA21FFF78F
:1043A0003BFB04F13C00FA21FFF736FB2571204668
:1043B000F8BD00BF38AD0000F0B51A4E05463068B4
:1043C0000A2489B0224600218A3004F037FC306884
:1043D00022460021943004F031FC00232A68009327
:1043E0000124019305F13C068DF815308DF8163047
:1043F000D7698DF814402846314622462346B847EF
:104400006B468DF8174043F8045B08AF17E90700C7
:1044100083E80700284631462246032300F006FAC7
:1044200009B0F0BDB888FF1FF0B589B004AA052314
:104430008DF81030036800920222002400F13C063F
:104440000192DF698DF8154031468DF81140032245
:10445000FE230546B8476B4608AF43F8044B17E9FF
:10446000070083E80700284631462246234600F02D
:10447000DDF909B0F0BD38B54C78CB6802341C4486
:104480000B780A2B0D46E4B201D18B7802E0142B95
:1044900003D14B7C1C44E4B202E00B2000F008FA8C
:1044A000E96800238B4205DAAA68D25C1444E4B2BE
:1044B0000133F7E7E043C0B238BD2DE9F0474E685D
:1044C0008D68089F0C46914600213246804628465A
:1044D0009A4604F0B3FB14222046002104F0AEFB00
:1044E0009DF8242066600A23B242A8BF3246A56028
:1044F000237084F801A084F80290E2601FB128467E
:10450000394600F0C1FE40462146FFF7B4FF207453
:10451000BDE8F0872DE9F8430446006DFCF796FFEF
:10452000012827DD206D0021FCF79AFFFF2805D127
:10453000206D0121FCF794FFFF2804D0206D01219C
:10454000FCF7B2FF16E0206DFCF780FF052811DDB7
:104550000221206DFCF784FF03210546206DFCF746
:104560007FFF0128064605D9206DFCF76FFFF31C7D
:10457000834201DB002533E0142365752375206D2C
:104580000421FCF76DFFA36984F82500B71E9F4244
:10459000A8BF1F4627620537FFB20525EBB2BB4215
:1045A0000BD22946206DD4F81C80FCF759FFA5F1E9
:1045B0000509013508F80900F0E73946206DFCF7D8
:1045C0004FFF04F11405074684F8240029462046CD
:1045D000FFF751FF8742206DB1D1311DFCF764FF19
:1045E0002846BDE8F88338B50546406D0A230B70B0
:1045F00003680C461B68FF219847686D0368FF211C
:104600001B689847686D617803681B689847686DF8
:10461000E168036802311B68C9B29847686DA178E8
:1046200003681B689847686DA1680368E2685B6867
:104630009847686D217C03681B68984738BD8B7864
:10464000032B11D1C86801280EDD89680B78022B75
:104650000AD918440238C0B2032805D8023BDBB29D
:104660000120CB5C13707047002070472DE9FF419B
:104670000446606D03689B68984758B1606D036895
:10468000DB689847C1B2206DFCF7CAFE4D4B1B6832
:10469000A360EEE72779002F4DD1E068FEF722FAFC
:1046A000002840F38B80E068FEF7D5F90DF10F028A
:1046B000011D2046FFF7C3FFD8B1434D9DF80F10F1
:1046C0002868FEF7CDFA002866D128689DF80F60AB
:1046D000FEF7BEFA86425FD0E0682D68FEF7BBF9B0
:1046E00041792846FEF7CBFA28449DF80F3080F830
:1046F0008A30206DFCF7D4FEE068FEF7ACF90023A9
:104700000546061D437631462046FFF76CFF6B7960
:10471000FE2B06D1012001F0E7FC20463146FFF7D1
:1047200062FF95F82430237113B9E068FEF7CEF9E3
:10473000244B1B681DE0012F2AD1E068DFF884803C
:10474000FEF789F905462046FFF7E4FED8F8002079
:10475000A368064678B995F82510D31A8B422DD94F
:104760006B7EEBB96F762046291DFFF73CFFD8F82A
:104770000030A36022E0144F71783868FEF77FFAAA
:1047800000280DDB3A68737C104480F8943007E011
:104790000C2000F08DF811E0E068FEF797F90DE0CD
:1047A000286830B10368009618351E6895E80E0039
:1047B000B047E068FEF78AF90023237104B0BDE832
:1047C000F08100BFD489FF1FB888FF1F38B5C568C6
:1047D000064B036004462DB12846FEF7EBF8284649
:1047E00003F003FD024B2360204638BD68AD000096
:1047F000C89B000010B50446FFF7E8FF204603F011
:10480000F4FC204610BDFFFF38B5074B036004469B
:10481000182003F0E8FC0F210546FA22FEF768F89D
:10482000E560204638BD00BF68AD0000F0B505ACBE
:104830001646059A44F8042B05460F46E8683946A3
:104840003246BDE8F040FEF7C4B8FFFFFB280CD0AD
:10485000FC2803D0FA2803D1054870470548704763
:10486000054B0130B3FBF0F070470448704700BFC0
:1048700010552200C0C62D0080841E00A0252600F1
:10488000400070478010EE38024B20EAE07053F889
:104890002000704790AD000040F26B135843000BAE
:1048A000704740F2DE735843B0FBF1F07047FFFFF2
:1048B00070B505462C46002C23DD012D12DD134E6C
:1048C000306878B100221346FF21FEF714F94FF447
:1048D0007A7001F009FC002130680A460B46FEF7A9
:1048E0000AF908E00A4B20261E604FF47A7001F0A6
:1048F000FBFB084B1E604FF47A7001F0F5FB013CA6
:10490000D9E74FF47A6001F0EFFBD3E7B888FF1FD7
:1049100084F00F4088F00F4070B51E4601FB00F494
:1049200012B104F011F902E0204604F04DF90C49EF
:104930000B6803B908600B4D0B680860C21A2B683E
:1049400013442B60084D2B681C442C6038B9074871
:104950000749324603F082FC1420FFF7A9FF70BD1F
:10496000DC88FF1FD888FF1FE088FF1FD091FF1F42
:10497000A0B90000054B1A6840F6B7339A420146C9
:1049800002D9034803F033BC704700BFD489FF1F2E
:10499000D091FF1F08B5084B1A6840F6B7339A420A
:1049A000014607D9054803F022FC0448BDE8084049
:1049B00003F03EBC08BD00BFD489FF1FD091FF1F8C
:1049C00008B5084B1A6840F6B7339A42014607D932
:1049D000054803F088FC0448BDE8084003F028BC03
:1049E00008BD00BFD489FF1FD091FF1F072910B554
:1049F0000C460BD872B600F05DFF62B60123A340EF
:104A00001840C0B240FA04F4E0B210BD002010BD5E
:104A100008B572B600F04EFF62B608BD08B572B6B2
:104A200000F05CFF62B608BD2DE9FF41234D2B6805
:104A3000642B07460C4690462E460DDD20496846FD
:104A400003F0B8FC6846FFF795FF684603F072FC78
:104A50002868FFF7B5FF2DE0072921D800F052FFA5
:104A60000028FBD072B6384600F024FF62B601235E
:104A700003FA04F418F0010F0CBF20EA0404044305
:104A8000E4B200F03FFF0028FBD072B63846214662
:104A900000F040FF62B633680133336001200AE062
:104AA0000849684603F086FC6846FFF773FF6846CE
:104AB00003F040FC002004B0BDE8F081E488FF1F53
:104AC000CCB9000021BA000070B50B4C2368642BF0
:104AD00005460E460EDC00F015FF0028FBD072B62E
:104AE0002846314600F016FF62B623680133236082
:104AF000012070BD002070BDE488FF1F70B50B4C15
:104B00002368642B05460E460EDC00F0FBFE0028F1
:104B1000FBD072B62846B1B200F016FF62B6236829
:104B200002332360012070BD002070BDE488FF1FA8
:104B300010B5044659B101210B20FFF7C5FF002134
:104B40000C20FFF7C1FF0D200221FFF7BDFF631E00
:104B5000DBB2FC2B05D821460E20BDE81040FFF744
:104B6000B3BF10BD08B500210220FFF7C7FF002129
:104B70001720FFF7C3FF002101221720FFF754FF82
:104B800001210A461720FFF74FFF41F244611A2026
:104B9000FFF7B4FF03210F20FFF796FF1020014617
:104BA000FFF792FF01211320FFF78EFF0121142050
:104BB000FFF78AFF03211520FFF786FF0321162048
:104BC000FFF782FF01200146BDE80840FFF7B0BFB4
:104BD00010B572B6094B0A4C01221A7020780221D6
:104BE00001F064F9074A084900231370074A13705B
:104BF0002078022201F054F862B610BD1D89FF1F13
:104C00000289FF1F1989FF1F814C0000EC88FF1FDC
:104C1000054B1A7810B51C4612B1044803F0D2FABD
:104C20000023237010BD00BF0189FF1F0489FF1FEF
:104C300010B5044603F0C6FA204610BD0B4B1A7897
:104C400010B51C460AB1FFF7E3FF094B094A1B6880
:104C5000591E914206D830225A4307480749013A63
:104C600003F09AFA0123237010BD00BF0189FF1FD2
:104C7000E888FF1F575555050489FF1FD94C0000D0
:104C800008B50F4B19781A46042309B10D4900E005
:104C90000D490B60127804230AB90A4A00E00A4A57
:104CA000136072B6094B187801F040F8084B0222E5
:104CB0001A70084B03221A70FFF7C0FF62B608BDD6
:104CC0001C89FF1F44F00F4048F00F400289FF1F6E
:104CD0001D89FF1F1889FF1F70B5404E3378012BC7
:104CE00003D1BDE87040FFF793BF3D4D2B78013BEA
:104CF000DBB22B70002B6FD13A4B1978042209B12B
:104D0000394900E039490A601A78344C82F00102CE
:104D10001A703278D2B2022A32D1354B1978354B1B
:104D200053F8313093F80002334B19780729C0B299
:104D300018D9012810D1314B31491A7808783149F6
:104D4000D2B2C0B2885419781422013191FBF2F02A
:104D500002FB1012D2B21A70FFF73AFF042333702D
:104D6000012319E01978C9B24C1CE4B21C70244B21
:104D70001C7800FA01F12143C9B219702A7070BD84
:104D80002378032B23D11C4B1A78072A06D9FFF767
:104D90001FFF0423237002232B7070BD144A154893
:104DA0001478174AE4B2117850F8340011F0010F6A
:104DB0004FF0010114BF80F8801080F800111178C5
:104DC000490811701A780132D2B21A70E3E72378D9
:104DD000042B04BF0123237070BD00BF1D89FF1F7A
:104DE0001889FF1F1C89FF1F44F00F4048F00F4037
:104DF0000289FF1FC4BA0000EC88FF1F1A89FF1F39
:104E00001989FF1FED88FF1F38B5104B1B78054629
:104E10000C4613B10320FFF74BFD1320012101F0D5
:104E200045F80B4B04221A6072B60A4A002313702D
:104E3000094A1370094B1D70094BB3FBF4F4094B7D
:104E40001C60FFF7C5FE62B638BD00BF1D89FF1F9D
:104E500048F00F401B89FF1F1A89FF1F0289FF1F9F
:104E600020A10700E888FF1F0B4B1A7810B58AB104
:104E70001A78012AFCD172B6084CFFF7C9FE2078D7
:104E800000F054FF2078022101F010F8024B0022BC
:104E90001A7062B610BD00BF1D89FF1F0289FF1F77
:104EA00072B6054B1878054B1B78C0B2DBB262B600
:104EB000C01A18BF012070471B89FF1F1A89FF1FE6
:104EC00010B5FFF7EDFF80B172B6084B08491A78AC
:104ED000D2B2885C19781422013191FBF2F402FB02
:104EE0001412D2B2C0B21A7062B610BD1B89FF1F75
:104EF000ED88FF1FF8B50746104E3578EDB2012D4D
:104F0000FAD172B60E4C207800F010FF03233370F4
:104F10000C4B1F700C4B00221A702078294600F0B1
:104F2000C5FF2278094B53F8323083F80051084B03
:104F300002221A70FFF782FE62B6F8BD1D89FF1FBC
:104F40000289FF1F1989FF1FEC88FF1FC4BA0000E8
:104F50001889FF1F04480549054A00230370802370
:104F6000437303F0E3BD00BF0489FF1F314C000011
:104F70006087FF1F084B1A6842F480721A604FF472
:104F8000A072013A7FF4FDAF1A689205FCD4202389
:104F9000013B7FF4FDAF7047005004402DE9F74F0F
:104FA0006A4E6B4B3268517E927E5C5C9D5CFF2C3E
:104FB000814601D0FF2D02D11120FFF779FC316825
:104FC000644A4B7E644F02EBC303586800230360BE
:104FD000897E624802EBC102614952681360614BED
:104FE000620013440B605F4B6A0013443B605E4BEE
:104FF0001A6842F020021A6001235C4A03FA05F5A0
:1050000003FA04F445EA04031360594B1A6822F0CA
:1050100080021A60574A1060574818608846B9F1F4
:10502000000F7AD0142001F05FF8FFF7A3FFD8F843
:10503000003052491B889BB2ADF80030BDF80030FB
:10504000BDF800204E4B92B20A601A603A684D4992
:10505000128892B2ADF80220BDF80220BDF80220FD
:1050600092B20A6048494FF00A0A0A609946FFF76F
:1050700081FFD8F80030414D1B88D9F800203868EE
:10508000404C9BB2ADF80430BDF80430BDF80410BC
:105090003E4B89B219602B684FF0060B42F20F7E2F
:1050A0000BFB02120EFB031342F21071B3FBF1F380
:1050B0002B6003889BB24FF0070CADF80630B2FBB3
:1050C000FCF2BDF80630BDF80600C9F800202268E1
:1050D0002F4B80B20BFB0202DFF8ACB01860DBF89C
:1050E00000300EFB0303B2FBFCF2B3FBF1F1052031
:1050F0000AF1FF3A2260CBF8001000F0F5FF1AF039
:10510000FF0AB4D11E4A336811682A688A1ADA6124
:105110002168DBF800208A1A1A62154B15491A68B3
:1051200022F080021A600A6842F420620A601A685B
:1051300042F0D2021A60174B80221A70A3F24B334E
:105140004FF400221A6003B0BDE8F08FB888FF1F4B
:1051500078BA0000C4BA00003C89FF1F00000303B6
:105160003889FF1F00510440388004400850044033
:10517000005004400450044080004D004089FF1F4F
:105180003489FF1F2C89FF1F2089FF1F3089FF1FD3
:105190002889FF1F53E400E02C4BF7B51A6812F47E
:1051A000805F1A680AD042F480521A60284B1A684D
:1051B000002001321A60FFF7F1FE45E042F40042A0
:1051C0001A60244B1B681B889BB2ADF80430BDF8F5
:1051D0000430BDF80420204B92B21A601F4B1C68AB
:1051E0004FF0060C07270CFB0424B4FBF7F41C60FB
:1051F0001B4B196842F20F7606FB012242F2107532
:10520000B2FBF5F21A60174B17491B681B889BB25B
:10521000ADF80630BDF80630BDF806309BB20B6025
:10522000124908680CFB0030B0FBF7F00860104929
:105230000F6806FB0733B3FBF5F30B600D490968F4
:10524000A21AC31ACA610B6203B0F0BD0050044039
:105250002489FF1F3889FF1F3089FF1F3489FF1FF2
:105260004089FF1F3C89FF1F2889FF1F2C89FF1FD2
:105270002089FF1FB888FF1F024B4FF400221A60DD
:10528000704700BF88E100E0844641EA000313F064
:1052900003036DD1403A41D351F8043B40F8043B3D
:1052A00051F8043B40F8043B51F8043B40F8043B00
:1052B00051F8043B40F8043B51F8043B40F8043BF0
:1052C00051F8043B40F8043B51F8043B40F8043BE0
:1052D00051F8043B40F8043B51F8043B40F8043BD0
:1052E00051F8043B40F8043B51F8043B40F8043BC0
:1052F00051F8043B40F8043B51F8043B40F8043BB0
:1053000051F8043B40F8043B51F8043B40F8043B9F
:1053100051F8043B40F8043B403ABDD2303211D33F
:1053200051F8043B40F8043B51F8043B40F8043B7F
:1053300051F8043B40F8043B51F8043B40F8043B6F
:10534000103AEDD20C3205D351F8043B40F8043B3F
:10535000043AF9D2043208D0D2071CBF11F8013B3D
:1053600000F8013B01D30B8803806046704700BF03
:10537000082A13D38B078DD010F003038AD0C3F112
:105380000403D21ADB071CBF11F8013B00F8013BF4
:1053900080D331F8023B20F8023B7BE7043AD9D3B3
:1053A000013A11F8013B00F8013BF9D20B78037088
:1053B0004B7843708B78837060467047F0B5304B04
:1053C0001B681B06FBD42F4B1B6813F08002F6D121
:1053D00072B62D4B1978002950D02C4908684F68B7
:1053E0008E68CD680C69384414313044096828440B
:1053F00020440844C0F34E00254940F400400860B2
:10540000C86A0F6B4E6B8D6BCC6B384440313044A7
:105410000968284420440844C0F34E001D4940F464
:105420000040086001F10811143151F8140C51F8D2
:10543000107C51F80C6C51F8085C51F8044C096868
:1054400038443044284420440844C0F34E001249F4
:1054500040F400400860C86A0F6B4E6B8D6BCC6BDC
:105460003844403130440968284420440844C0F39B
:105470004E000A4940F4004008601A7062B6F0BD60
:1054800024B0034024B00B404589FF1F38B00340CF
:105490002CB0034030B003402CB00B4030B00B4078
:1054A00010B5204B2048214960221A70E1225A7021
:1054B0001F4B204A1C78204B082C01D1012402E00C
:1054C0000A2C03D139240460132005E00C2C0CBFF6
:1054D00035243D2404601220086014601860174BC6
:1054E00017491B78174A03B101230B601360164B51
:1054F000164A1978164B012901D880210BE004299E
:1055000001D8842107E0082901D8852103E010296A
:1055100094BF86218721116019600E4B01221A70F9
:1055200010BD00BF0040074008B003400CB003406E
:105530006887FF1F08B00B400CB00B404889FF1F65
:1055400020B0034020B00B406987FF1F24B0034008
:1055500024B00B404589FF1F0C2804D9102828BF10
:105560001020102307E00A2804D8092834BF082394
:105570000A2300E00C23094AD9B2081A1070084A1D
:105580001078834208D0074B11701B7813B1064B7B
:1055900000221A60FFF784BF704700BF4489FF1FD5
:1055A0006887FF1F4589FF1F24B0034010B5114BCA
:1055B0001B7804460BB1FFF701FF012C0E4A01D8FE
:1055C000002302E0042C02D8042313600EE0082C10
:1055D00003D805231360082308E0102C03D8062302
:1055E0001360102302E0072313602023034A137083
:1055F00010BD00BF4589FF1F24B003406987FF1F0E
:105600000D2838B50FD9172801D80E380AE0A0F1B7
:105610001A03052B01D8093804E0A0F12203062B58
:1056200047D81838C0B2244B1C5C244B1B780BB1F4
:10563000FFF7C4FE210614D472B6214B214D1C6025
:1056400001232B7062B672B61D4B1B681A0601D57A
:105650001D4B1FE02B78002BEFD062B602F0D6FE78
:10566000F1E772B6194B1A4D1A6814F0400F14BFC7
:1056700022F0100242F010021A60164B04F03F02B2
:105680001A6001232B7062B672B6124B1B681B06A0
:1056900008D5114B186800232B7062B60F4B1B788E
:1056A000184138BD2B78002BDCD062B602F0AEFE7C
:1056B000EAE7002038BD00BF9ABA00004589FF1F05
:1056C00000B003404789FF1F10B003400CB00B40EF
:1056D0004689FF1F00B00B4010B00B404489FF1FEC
:1056E0000D2810B50FD9172801D80E380AE0A0F1FF
:1056F0001A03052B01D8093804E0A0F12203062B78
:1057000027D81838C0B2134B1C5C134B1B780BB155
:10571000FFF754FE230607D472B6104B44F0400442
:105720001C6001220E4B12E072B60E4B1A6814F088
:10573000400F14BF22F0100242F010021A6004F071
:105740003F04094B44F040041C60084B01221A70CE
:1057500062B610BD9ABA00004589FF1F00B0034031
:105760004789FF1F0CB00B4000B00B404689FF1F5C
:105770000D280FD9172801D80E380AE0A0F11A0316
:10578000052B01D8093804E0A0F12203062B26D806
:105790001838C0B2134B1B56002B08DB124B1B688A
:1057A00013F0800F114B12D072B6114A07E0114B63
:1057B0001B6813F0800F104B09D072B60F4A1068A7
:1057C00000221A7062B60E4B1B78184170471B7886
:1057D000002B14BF4FF0FF306FF001007047002026
:1057E000704700BF9ABA000000B003404789FF1F0E
:1057F00010B0034000B00B404689FF1F10B00B40B3
:105800004489FF1F084B1A6842F480521A60074B04
:105810001A78074B0AB1802200E0C0221A70054BAB
:1058200080F30C00188070472C8004404889FF1FCB
:1058300021C00C4000C00C40024B1B78DB07FBD59D
:10584000704700BF010002407FB5174B6A4603F165
:1058500010056E4618685968144603C40833AB42F5
:105860002246F7D1114B1A7812F0020F1D4612D0C2
:1058700080229A7133229A7203225A7272B60C4CA9
:1058800046F001062046B04762B6237813F0700355
:1058900001D0237006E044F621632A78D20701D4B0
:1058A000013BFAD104B070BDB2BA00000100024061
:1058B00000000240B0F5006F10B5044609D2064B57
:1058C0001B78DB0701D4FFF7BFFF04F1A054207859
:1058D00010BD002010BD00BF0100024040F2FE7369
:1058E000984210B5044609D8054B1B78DB0701D454
:1058F000FFF7AAFF04F1A054208810BD002010BDBE
:1059000001000240024B187800F00100704700BF10
:1059100001000240B0F5006F38B504460D460FD2C5
:10592000084B1B78DB0701D4FFF78EFF04F1A0546E
:105930002378AB4204D02570BDE83840FFF77CBF28
:1059400038BD00BF0100024038B540F2FE739842F6
:1059500004460D461ED8104B1B78DB0701D4FFF719
:1059600073FF14F0010F04F1A05404D12388AB425B
:1059700010D025800AE02378AB4202D02570FFF7D3
:105980005BFF63782D0AAB4204D06570BDE83840F8
:10599000FFF752BF38BD00BF01000240024B1A683A
:1059A00001321A60704700BFD489FF1F08B50B4C45
:1059B0002368580301D501F013FD2368590501D56B
:1059C00000F03CFE23681A0501D501F017F92368A1
:1059D000DB04ECD501F080FBE9E700BF3480044034
:1059E00008B5FFF7E3FFFFFF014B10221A80704755
:1059F000002005407047FFFF024A136818441060FA
:105A0000184670476C87FF1F002070474FF0FF302B
:105A100070474FF0FF307047FEE7FFFFEFF313834F
:105A20009BB9EFF3108098B9EFF3058323B10F2BE7
:105A300004D9084A985C01E04FF48070EFF31183B9
:105A40003BB1834238BF184670474FF0FF30704774
:105A500018467047F0E300E01F4B10B51C681C604F
:105A6000E00304D51D4B1A680AB11B689847A103CF
:105A700004D51A4B5A680AB15B689847E20704D507
:105A8000164B1A6C0AB11B6C9847A30704D5134B2D
:105A90005A6C0AB15B6C9847200704D50F4B9A6C7F
:105AA0000AB19B6C9847610704D50C4BDA6C0AB1BC
:105AB000DB6C9847220304D5084B5A6E0AB15B6E23
:105AC0009847630306D5054BD3F8802012B1D3F86D
:105AD0008030984710BD00BFA0A004404C89FF1F34
:105AE0002C4B10B51C681C60200704D52A4B5A6A41
:105AF0000AB15B6A9847E10604D5274B9A6A0AB156
:105B00009B6A9847620604D5234BDA6A0AB1DB6ABE
:105B10009847230604D5204B1A6B0AB11B6B984794
:105B2000A00604D51C4B5A6B0AB15B6B9847E10782
:105B300004D5194BDA6B0AB1DB6B9847A20704D581
:105B4000154B9A6D0AB19B6D9847630704D5124BAC
:105B5000DA6D0AB1DB6D9847A00504D50E4BDA6EFD
:105B60000AB1DB6E9847E10504D50B4B1A6F0AB1F9
:105B70001B6F9847620504D5074B5A6F0AB15B6FDC
:105B80009847230504D5044B9A6F0AB19B6F984739
:105B900010BD00BFA0B004404C89FF1F1E4B10B5C4
:105BA0001C681C60E00704D51C4B9A680AB19B680E
:105BB0009847210604D5194B5A690AB15B69984781
:105BC000E20604D5154B9A690AB19B6998476307A9
:105BD00004D5124BDA690AB1DB699847200704D56E
:105BE0000E4B1A6A0AB11B6A9847A10704D50B4BE2
:105BF0009A6B0AB19B6B9847A20604D5074B1A6DA6
:105C00000AB11B6D9847630604D5044B5A6D0AB15F
:105C10005B6D984710BD00BFA0C004404C89FF1FBA
:105C2000114B10B51C681C60E00404D50F4BDA68FA
:105C30000AB1DB689847A10404D50C4B1A690AB174
:105C40001B699847A20604D5084B1A6E0AB11B6E51
:105C50009847E30606D5054BD3F8842012B1D3F854
:105C60008430984710BD00BFA09004404C89FF1FAE
:105C7000094B10B51C681C60A20704D5074B9A6E2F
:105C80000AB19B6E9847E30704D5044BDA6F0AB15B
:105C9000DB6F984710BD00BFA0D004404C89FF1FA8
:105CA000212830B531D8042A2FD8DFE802F00709BF
:105CB000050B03000B2306E00A2304E0082302E09F
:105CC0000C2300E00923114A114D02EBC002546875
:105CD000104AC2F89C51104DC2F8A0510F4DC2F8A5
:105CE000A4510F4DC2F8A8510E4DC2F8AC5172B676
:105CF00022680D4D22F47022226042F0807242EA46
:105D0000034345F82010236062B630BDC4BA0000DA
:105D1000215C00000082FF1F595A0000E15A000078
:105D20009D5B0000715C00004C89FF1F094B03EB79
:105D3000C0035A6872B6136823F0877323F4803364
:105D400043F080731360044B002243F8202062B6B6
:105D5000704700BFC4BA00004C89FF1F044B0549BF
:105D600000221A600A60044A106010221A6070470C
:105D700014D0034004D0034000D003402DE9F0418B
:105D800005460E4608462E4902F062FE2D4B0028BD
:105D900047F6122814BF0227012708BF984600249F
:105DA00028FA04F002F05EFC4FF05E5102F0B2FC03
:105DB0000146304602F060FE10B90134072CEFD1E5
:105DC00028FA04F002F04EFC314602F057FD4FF085
:105DD0007C5102F095FB02F089FE4FF6FF7398426A
:105DE00028BF1846EB1E012B06D8174B1749002277
:105DF0001A600A60164A1BE0A5F10903012B06D9B7
:105E0000A5F11403032B02D96B1F012B06D8114BEC
:105E1000114900221A600A60104A09E0202D01D0C1
:105E2000192D0BD10E4B0F4900221A600A600E4A41
:105E300004F0070444EAC70710601F60BDE8F08162
:105E4000001BB740006CDC0200900340049003404C
:105E50000890034000800340048003400880034012
:105E600000800B4004800B4008800B40212810B5B7
:105E700018D80D4A52F8303093F880423CB10122D4
:105E800011B183F8802010BD83F8002110BD02EB12
:105E9000C00043681A6811B142F0030201E022F029
:105EA00002021A6010BD00BFC4BA0000212816D833
:105EB0000B4A02EBC00301295B6852F8302004D181
:105EC00082F880124FF4A27208E0002082F880026B
:105ED00011B94FF4807201E040F203121A6070476A
:105EE000C4BA0000282838B5604A04460B4611D1D0
:105EF00012780B2A04D8C2F10C0201FA02F304E072
:105F00000C2A1CBF0C3A41FA02F31846BDE838408F
:105F1000FFF778BC11780125002B05FA01F2D8BFF4
:105F2000002102DD934205D32946FFF79FFF20465B
:105F3000294697E00338C2B2012A01D84C4A06E04C
:105F4000202C01D0192C01D14A4A00E04A4A12689B
:105F500002FB0332CA401D287BD8DFE800F0575F00
:105F60004E337A7A212A7A7A7A7A7A7A7A7A7A3CEB
:105F7000450F187A707A7A7A7A7A7A673F4B1A6084
:105F800003F5973340F2444203F5FA735FE03C4B6C
:105F90001A6003F5973340F2444203F5F87356E074
:105FA000384B1A6003F5973340F2444203F5F67319
:105FB0004DE0354B1A6003F5973340F2444203F548
:105FC000F47344E0314B1A6003F59F3340F24442CE
:105FD00003F5F0733BE02E4B1A6003F59F3340F25C
:105FE000444203F5EE7332E02A4B1A6003F59F3307
:105FF00040F2444203F5EC7329E0274B1A6003F5A5
:106000009F3340F2444203F5EA7320E0234B1A60C9
:1060100003F580334FF45172203318E0204B1A609F
:1060200003F580334FF451721C3310E01D4B1A609E
:10603000A3F5DB234FF45172A3F5F96307E01A4B84
:106040001A60A3F5DB234FF45172A3F2CC731A60EC
:1060500038BD7F2B2046D4BF00210121FFF706FF6A
:1060600020460121BDE83840FFF720BF7087FF1FA1
:106070000890034008800B400880034010800340D4
:106080001880034020800340288003403080034074
:106090003880034040800340488003401090034014
:1060A0001890034010800B4018800B4072B60B4BC9
:1060B0000B491A680B4B1B68096862B6490102D587
:1060C000322A88BF0133C2F5BB326021FF32B2FBF6
:1060D000F1F24FF47A7000FB0320704718E000E003
:1060E00004ED00E0D489FF1F38B50446FFF7DEFF5A
:1060F000054624B938BD013C0AD005F57A75FFF78D
:10610000D5FF401BB0F57A7FF5D202F07FF9F6E7B4
:1061100038BDFFFF1F4B4FF4000210B51A604FF05F
:1061200080721A604FF000721A604FF080621A603D
:106130004FF000621A60184B184A194C00204BF6B9
:10614000FF71186059602823136093601361936195
:1061500013629362136393630922226004F58054EF
:10616000043420606160A360236144F8042C04F5CA
:10617000FE2420600B4801600B490B608B600B4BC9
:106180001A60FFF78DF9FA20FFF7AEFFBDE8104067
:1061900001F024BC08E100E0048003400C800340CF
:1061A0000080034008800B400C800B4000800B40B7
:1061B000194B1A6842F480621A60184A002313804F
:1061C000174A1380174A1370174A1370174A13702F
:1061D000174B40F213321A604FF451725A60154B4C
:1061E000C0F344321A70C0F347125A7002210422DD
:1061F00000F01F0098729A70D9745A7588221A7428
:106200003C22DA700C4B40226FF44A711A700B4436
:106210004FF400521A60704734800440608BFF1FB7
:10622000DE89FF1F688BFF1F628BFF1FDC89FF1F4A
:1062300040A0044000A006402DE400E0134A9378FB
:1062400000F0030103F0EC030B43410748BF43F0A8
:106250001003937000F00F03042B0C4903D18B79CA
:1062600043F040038B715379C20603F0EF03074AF2
:1062700048BF43F0100353719379810603F0EF0395
:1062800048BF43F010039371704700BF00A0064061
:1062900008B5114B1B685B0500D408BD0F4B1A787D
:1062A00002F0FF0312B102F0B1F8F7E70C4A4FF425
:1062B000005111600B4A0C49D37040F203120A607E
:1062C0004A600A4A13800A4A13800A4B1B680BB1C2
:1062D00001221A7008BD00BF34800440DC89FF1F12
:1062E00084E100E000A0064040A00440608BFF1F56
:1062F000DE89FF1FD889FF1F38B50446094B1B787C
:1063000003F0FF05002BF9D120460121FFF7CEFD58
:1063100020462946FFF7AAFD034B53F83420034BD0
:106320001A6038BDDC89FF1FC4BA0000648BFF1FF0
:106330000D4A38B5146814F480624FF0000410D090
:1063400021280A4D0AD80A4A012152F830302B6020
:10635000FFF7ACFD2B681C70012038BD2C60204677
:1063600038BD104638BD00BF34800440D889FF1FB7
:10637000C4BA00000E4B1B6813F4806316D01228B9
:106380000C4B03D140F202310B4A04E0142809D12E
:106390000A4A40F2023111605A7B42F001025A73FC
:1063A000012070475A7B02F0FE025A7300207047AA
:1063B0003480044000A006400CA0044014C00440F7
:1063C000F8B51D4B1B685A05064633D51B4B1B6899
:1063D0000BB101221A701A4B1C780134802C1F4615
:1063E00028BF0024174D2B78A34218D1FFF716FBC6
:1063F00040280FDC144A13791B06F3D52B78134978
:106400000133802B28BF0023C95CDBB2C9B2D17134
:106410002B70E7E7FF28E5DD01F0F8FFE2E70B4B23
:10642000F6B21E550A4B01221A70074BE4B2BC2289
:106430003C70DA70F8BD00BF34800440648BFF1FED
:10644000688BFF1F628BFF1F00A00640E089FF1FC3
:10645000DC89FF1F274B1B685A052DE9F0470746CB
:106460008A4644D5244B1B680BB101221A703D4665
:1064700007EB0A039D4237D2DFF890801F4E98F851
:10648000004096F800900134802C28BF00245FFA69
:1064900089F9A1451DD11A4BBC22DA70FFF7BEFA6B
:1064A00040280FDC164A13791B060FD5337815499F
:1064B0000133802B28BF0023C95CDBB2C9B2D17184
:1064C000337003E0FF2801DD01F0A0FF33784B4576
:1064D000E4D00C4B15F8012B1A550B4B0122E4B2FA
:1064E0001A7088F80040C3E7054BBC22DA70BDE89B
:1064F000F08700BF34800440648BFF1F628BFF1F56
:1065000000A00640E089FF1FDC89FF1F688BFF1F8A
:1065100008B5034B1B7813B101F078FFF9E708BD0C
:10652000DC89FF1F064A074B1B781078DBB2C0B22C
:1065300083422CBF7F3000F1FF30C01A704700BF8C
:10654000628BFF1F688BFF1F054B1888054B1B884C
:1065500080B29BB2984238BF00F58070C01A704775
:10656000608BFF1FDE89FF1F114B12491A880B88B1
:1065700092B29BB29A4210B516D00133B3F5807F28
:1065800028BF00230C489CB2C05C0C800B490968F2
:10659000C0B259B19A4238BF02F58072D31A1A2B91
:1065A00004DC00230B7010BD4FF0FF3010BD00BFA6
:1065B000608BFF1FDE89FF1F608AFF1FD889FF1FC6
:1065C000094B1A88094B1B8892B29BB29A4208D099
:1065D0000133B3F5807F28BF0023054AD05CC0B2E9
:1065E00070474FF0FF307047608BFF1FDE89FF1F41
:1065F000608AFF1F0C4B1B685B0514D50B4BDA78C8
:1066000002F0CB02DA7040225A74DA7842F0340297
:10661000DA70074B1A88074B92B21A80064B1B6838
:106620000BB100221A7070473480044000A006406D
:10663000DE89FF1F608BFF1FD889FF1F30B53D4BE0
:106640001A7912F0300F32D072B69A7D02F0FF0044
:1066500022B9DA7940225A7462B628E062B6364A24
:106660003649138809889BB289B21446314AD579D4
:106670005A1CB2F5807F28BF00228A42EDB202D0B8
:106680002F4B9D541346421E12F0FF00EED19AB2DA
:1066900022802C4A126852B18B4236BFC1F58071FC
:1066A000C1EB03035B18272BC4BF01231370214BDD
:1066B000D978C9B20D0620D51B791C061DD5224BF1
:1066C000224A1D781378EDB2DBB21046AB420CD0F3
:1066D000184A0133802B14791D4C28BF0023E45C39
:1066E000E4B2D471127D072AF0D9DBB20370114BEA
:1066F0001A79100644BF7C22DA700E4B9A7C52073E
:1067000006D5144A10780130C0B2107004229A7471
:106710004B060ED5074B1A7912F0400F194608D0D8
:106720000D4B00221A700D4B1B6803B11A703C23ED
:10673000CB7030BD00A00640608BFF1FDE89FF1FBD
:10674000608AFF1FD889FF1F688BFF1F628BFF1FA6
:10675000E089FF1FEC91FF1FDC89FF1F648BFF1F87
:106760001D4B1A6842F400621A601C4A0023138011
:106770001B4A13801B4A13701B4A13701B4A137069
:106780001B4B40F213321A604FF451725A60194B8E
:10679000C0F344321A70C0F347125A7000F01F0061
:1067A0000422022198729A70D9745A7588221A7438
:1067B0003C22DA709A7842F0A0029A709A7902F03C
:1067C000DF029A710C4B40221A70A3F22B334FF464
:1067D00000421A60704700BF34800440748DFF1F70
:1067E000728BFF1F7C8DFF1F768DFF1F708BFF1F2D
:1067F0000CB0044000B006402FE400E0134A937848
:1068000000F0030103F0EC030B43410748BF43F0E2
:106810001003937000F00F03042B0C4903D18B7904
:1068200043F040038B715379C20603F0EF03074A2C
:1068300048BF43F0100353719379810603F0EF03CF
:1068400048BF43F010039371704700BF00B006408B
:1068500008B5114B1B681B0500D408BD0F4B1A78F7
:1068600002F0FF0312B101F0D1FDF7E70C4A4FF43B
:10687000004111600B4A0C49D37040F203120A60C8
:106880004A600A4A13800A4A13800A4B1B680BB1FC
:1068900001221A7008BD00BF34800440708BFF1FB6
:1068A00084E100E000B006400CB00440748DFF1F8E
:1068B000728BFF1F6C8BFF1F38B50446094B1B788A
:1068C00003F0FF05002BF9D120460121FFF7EEFA76
:1068D00020462946FFF7CAFA034B53F83420034BEE
:1068E0001A6038BD708BFF1FC4BA0000788DFF1F7F
:1068F0000D4A38B5146814F400624FF0000410D04B
:1069000021280A4D0AD80A4A012152F830302B605A
:10691000FFF7CCFA2B681C70012038BD2C60204694
:1069200038BD104638BD00BF348004406C8BFF1F5B
:10693000C4BA00000B4B1B6813F4006310D0172877
:10694000094B09D1094A40F2023111605A7B42F0E9
:1069500001025A73012070475A7B02F0FE025A73FB
:10696000002070473480044000B0064008B0044066
:10697000F8B51F4B1B681A05064638D51D4B9A798A
:1069800042F020029A711C4B1B680BB101221A7055
:106990001A4B1C780134802C1F4628BF0024184D48
:1069A0002B78A34218D1FFF739F840280FDC114AA1
:1069B00013791B06F3D52B7812490133802B28BF9E
:1069C0000023C95CDBB2C9B2D1712B70E7E7FF28A5
:1069D000E5DD01F01BFDE2E70A4BF6B21E550A4B5E
:1069E00001221A70034BE4B2BC223C70DA70F8BD8D
:1069F0003480044000B00640788DFF1F7C8DFF1F5F
:106A0000768DFF1F748BFF1F708BFF1F294B1B6838
:106A10001A052DE9F04707468A4649D5264B9A794B
:106A200042F020029A71254B1B680BB101221A70AB
:106A30003D4607EB0A039D4237D2DFF89080204E97
:106A400098F8004096F800900134802C28BF00246C
:106A50005FFA89F9A1451DD1174BBC22DA70FEF708
:106A6000DDFF40280FDC144A13791B060FD533785D
:106A700014490133802B28BF0023C95CDBB2C9B2A3
:106A8000D171337003E0FF2801DD01F0BFFC3378E2
:106A90004B45E4D00B4B15F8012B1A550A4B01223C
:106AA000E4B21A7088F80040C3E7034BBC22DA70E6
:106AB000BDE8F0873480044000B00640788DFF1FA9
:106AC000768DFF1F748BFF1F708BFF1F7C8DFF1F48
:106AD00008B5034B1B7813B101F098FCF9E708BD2A
:106AE000708BFF1F064A074B1B781078DBB2C0B2D1
:106AF00083422CBF7F3000F1FF30C01A704700BFC7
:106B0000768DFF1F7C8DFF1F054B1888054B1B885A
:106B100080B29BB2984238BF00F5C070C01A70476F
:106B2000748DFF1F728BFF1F114B12491A880B883F
:106B300092B29BB29A4210B516D00133B3F5C07F22
:106B400028BF00230C489CB2C05C0C800B4909682C
:106B5000C0B259B19A4238BF02F5C072D31A1A2B8B
:106B600004DC00230B7010BD4FF0FF3010BD00BFE0
:106B7000748DFF1F728BFF1FF48BFF1F6C8BFF1F29
:106B8000094B1A88094B1B8892B29BB29A4208D0D3
:106B90000133B3F5C07F28BF0023054AD05CC0B2E3
:106BA00070474FF0FF307047748DFF1F728BFF1FCF
:106BB000F48BFF1F0C4B1B681B0514D50B4BDA78AD
:106BC00002F0CB02DA7040225A74DA7842F03402D2
:106BD000DA70074B1A88074B92B21A80064B1B6873
:106BE0000BB100221A7070473480044000B0064098
:106BF000728BFF1F748DFF1F6C8BFF1F30B53E4BD8
:106C00001A7912F0300F32D072B69A7D02F0FF007E
:106C100022B9DA7940225A7462B628E062B6374A5D
:106C20003749138809889BB289B21446324AD5790C
:106C30005A1CB2F5C07F28BF00228A42EDB202D0B2
:106C4000304B9D541346421E12F0FF00EED19AB213
:106C500022802D4A126852B18B4236BFC1F5C071F5
:106C6000C1EB03035B18272BC4BF01231370224B16
:106C7000D978C9B20A0620D51B791D061DD5234B2C
:106C8000234A1D781378EDB2DBB21046AB420CD02C
:106C9000194A0133802B14791E4C28BF0023E45C71
:106CA000E4B2D471127D072AF0D9DBB20370124B23
:106CB0001A79140644BF7C22DA700F4B9A7C500775
:106CC00006D5154A10780130C0B2107004229A74AB
:106CD000490610D5084B1A7952060CD50F4A0021E7
:106CE00011700F4A126802B111709A7902F0DF0236
:106CF0009A713C22DA7030BD00B00640748DFF1FDF
:106D0000728BFF1FF48BFF1F6C8BFF1F7C8DFF1F8F
:106D1000768DFF1F748BFF1FD488FF1F708BFF1FA2
:106D2000788DFF1F174B1A6842F480521A60164A7A
:106D300000231380154A1380154A1380154A1380C7
:106D4000154A1370154A40F2133111604FF4517116
:106D50005160134AC0F344311170C0F3471100F081
:106D60001F0051709072937013742C23D3700D4BCD
:106D700040226FF44B711A700B444FF400321A60CA
:106D8000704700BF348004408890FF1F868DFF1F2E
:106D90009090FF1F8A90FF1F848DFF1F08C0044042
:106DA00000C0064031E400E0134A937800F003018C
:106DB00003F0EC030B43410748BF43F0100393700B
:106DC00000F00F03042B0C4903D18B7943F04003EF
:106DD0008B715379C20603F0EF03074A48BF43F0B3
:106DE000100353719379810603F0EF0348BF43F01A
:106DF00010039371704700BF00C0064008B5114BE7
:106E00001B68DB0400D408BD0F4B1A7802F0FF03A7
:106E100012B101F0FBFAF7E70C4A4FF400311160B0
:106E20000B4A0C49D37040F203120A604A600A4AC6
:106E300013800A4A13800A4B1B680BB101221A7097
:106E400008BD00BF34800440848DFF1F84E100E052
:106E500000C0064008C004408890FF1F868DFF1FB9
:106E6000808DFF1F38B50446094B1B7803F0FF05E2
:106E7000002BF9D120460121FFF718F820462946BA
:106E8000FEF7F4FF034B53F83420034B1A6038BD70
:106E9000848DFF1FC4BA00008C90FF1F0D4A38B5C7
:106EA000146814F480524FF0000410D021280A4DC9
:106EB0000AD80A4A012152F830302B60FEF7F6FF5B
:106EC0002B681C70012038BD2C60204638BD104650
:106ED00038BD00BF34800440808DFF1FC4BA00005D
:106EE0000B4B1B6813F4805310D00E28094B09D1AB
:106EF000094A40F2023111605A7B42F001025A7392
:106F0000012070475A7B02F0FE025A73002070473E
:106F10003480044000C0064004C00440F8B51F4B54
:106F20001B68DA04064638D51D4B1B680BB10122DD
:106F30001A701C4B1C88A4B20134B4F5C07F1F46E4
:106F400028BF0024184D2B889BB2A3421AD1FEF70C
:106F500065FD402811DC154A13791B06F2D52B88F4
:106F600013499BB20133B3F5C07F28BF0023C95C2E
:106F70009BB2C9B2D1712B80E4E7FF28E2DD01F0BA
:106F800045FADFE70A4BF6B21E550A4B01221A708A
:106F9000064BA4B2AC223C80DA70F8BD34800440C9
:106FA0008C90FF1F9090FF1F8A90FF1F00C006402B
:106FB000888DFF1F848DFF1F38B504464518AC42ED
:106FC00004D014F8010BFFF7A9FFF8E738BDFFFF65
:106FD00008B5034B1B7813B101F018FAF9E708BDA7
:106FE000848DFF1F064A074B1B8810889BB280B216
:106FF00083422CBF00F27F1000F1FF30C01A7047AF
:107000008A90FF1F9090FF1F054B1888054B1B8827
:1070100080B29BB2984238BF00F5C070C01A70476A
:107020008890FF1F868DFF1F114B12491A880B880D
:1070300092B29BB29A4210B516D00133B3F5C07F1D
:1070400028BF00230C489CB2C05C0C800B49096827
:10705000C0B259B19A4238BF02F5C072D31A1A2B86
:1070600004DC00230B7010BD4FF0FF3010BD00BFDB
:107070008890FF1F868DFF1F088FFF1F808DFF1FC9
:10708000094B1A88094B1B8892B29BB29A4208D0CE
:107090000133B3F5C07F28BF0023054AD05CC0B2DE
:1070A00070474FF0FF3070478890FF1F868DFF1F9D
:1070B000088FFF1F054B1A88054B92B21A80054BAB
:1070C0001B680BB100221A70704700BF868DFF1F2E
:1070D0008890FF1F808DFF1F10B5314B1A799206E3
:1070E00023D5304AD87913882F499BB201330988B8
:1070F000B3F5C07F28BF002389B28B42C0B203D052
:107100002A49C85499B21180294A116869B1294A9B
:10711000128892B2934236BFC2F5C072C2EB03032B
:107120009B18272BC4BF01230B701D4AD178C9B20D
:107130000C0618D51379180615D51F4B1D481C8849
:107140000388A4B29BB29C4202D16C23D3700AE0A4
:107150000133B3F5C07F28BF0023184CE45C9BB219
:10716000E4B2D47103800E4B9A7C520706D5144AC0
:1071700010780130C0B2107004229A744B060ED5FC
:10718000074B1A7912F0400F194608D00D4B002218
:107190001A700D4B1B6803B11A702C23CB7010BDF5
:1071A00000C006408890FF1F868DFF1F088FFF1FBD
:1071B000808DFF1F8A90FF1F9090FF1F888DFF1FFB
:1071C000ED91FF1F848DFF1F8C90FF1F21282BD86E
:1071D000164B1B5CFF2B27D0154A02EBC000002189
:1071E00042681160134A106840F020001060124A93
:1071F00001201160114998400860114841F8040CC1
:10720000104911604FF4A07101397FF4FDAF11688E
:107210008905FCD42022013A7FF4FDAF0A4A1BB253
:1072200032F8130080B2704700207047D4BB0000D2
:10723000C4BA0000388004400050044008500440A4
:107240000000020380014A0000510440F0B50C4BDD
:107250000C4C1A7842F0020504EBC50682F00102DC
:10726000706009481A700678002E0CBF8827C8275E
:1072700086F0010647EA0141067044F83510F0BD7A
:10728000FC90FF1F0080FF1F7491FF1F431E032B04
:1072900010B510D872B6094A52F8230048B14168B7
:1072A00042F82310064A018832F81340611A22F886
:1072B000131062B610BD002010BD00BFEC90FF1F80
:1072C000EE91FF1F013803280AD872B6054B53F818
:1072D0002030002013B101305B68FBE762B67047D5
:1072E000002070474091FF1F10B572B60123174A66
:1072F0001A4412F8012C12071CD59900144A52F8AE
:1073000031402CB902EB431308305860114B09E0AF
:1073100041F0010152F8314064B902EBC103083079
:1073200058600D4B42F831300C4B1A78013A1A7004
:1073300062B610BD0133052BD9D162B6074B0022CE
:107340001A70BDE8104000F0A7BB00BF28BD0000C8
:107350000080FF1F88004000C80040006A91FF1FA6
:10736000431E032B30B532D8194A400140F01000BB
:10737000104472B6174CE25C032A09D8DFE802F029
:10738000160218050830022213E00830042210E02B
:107390001148124A50F8234014B940F8231002E073
:1073A00052F82300416042F823100FE0032200E06E
:1073B0000522E25410F0080F01F108030A88436027
:1073C0000CBF8823C82343EA0243036062B630BD82
:1073D0000080FF1FA890FF1F4091FF1F5091FF1FCB
:1073E0002DE9F84FAB4F3C78E4B214F0040F3D4662
:1073F00019D0A94B1B78A3B1A84A117801F0FF035B
:1074000021B1013BDBB2137003B900BEA44A11786D
:1074100001F0FF0329B1013BDBB213700BB900F09F
:107420004FFC04233B7004F0080303F0FF02002B21
:1074300000F067829B4B9C4C1A78D2B215094FEA38
:10744000920840F0E48104EBC803596854F83830DE
:10745000C3F38303013B0C2B00F2D681DFE813F06A
:1074600095019501D401D401D401D401D401D401F2
:10747000B001D401D401D4010D008C4D0A684B68D1
:107480008B486B6001218B4B44F838302A60DFF861
:107490005082017092B240F2816000238242C8F8AB
:1074A00000302361A36117D8B2F5D06F80F01E8140
:1074B000B2F5817F00F0CF8006D8802A00F0BA8034
:1074C000822A00F0BB8031E140F202339A4200F0A0
:1074D000D180B2F5A06F1CE042F22100824200F0A0
:1074E00051810ED8B2F5086F00F09E80B2F5106F92
:1074F00040F01C81684B6C4EAA781A7006F1800926
:107500000AE042F221218A4200F0088142F221334E
:107510009A4200F00F8109E1336A1B0603D5706AB5
:10752000083800F0B9FA08364E45F5D10026B146C4
:10753000DFF8B0A156F80A0028B1D0F804B000F086
:10754000ABFA5846F8E74AF806005B4BDFF898A11B
:10755000F05056F80A0028B1D0F804B000F09CFAB8
:107560005846F8E7554B4AF80600F050544B23F8BC
:107570001900544B19F80320023A032A08D8DFE80F
:1075800002F002040204002200E0012203F80920B4
:1075900009F10109B9F1040F06F10406C8D14A4BFB
:1075A00000221A7001269A46484A494B3244334415
:1075B00012F8012C9B0012F0080F1A704FEA86098E
:1075C00025D000F04BFA38B104EB46130830586070
:1075D000404B44F8393006E09AF8003044F839005E
:1075E00001338AF8003000F039FA49F0010338B16C
:1075F00004EBC302083050602E4A44F8332006E002
:1076000044F833009AF8003001338AF8003049F02A
:107610000202013649F003090023052E44F83230F6
:1076200044F83930C0D186E01B4B2B4C1B782370BB
:107630000B4683E0284C237063707EE0AA88042AFE
:1076400074D8254C920023706370244B9B5C9E077A
:1076500073D5217071E0AA8802F07F02042A65DCEC
:107660006B88002B62D191001C4A0A44117821F0EA
:10767000020159E0AA8802F07F02042A56DC6B88D6
:10768000002B53D19100154A0A44117841F00201B0
:107690004AE000BF802007407391FF1FFD90FF1F4D
:1076A0007591FF1F902007400080FF1F6091FF1F12
:1076B0007491FF1FC80040009890FF1F5091FF1F5A
:1076C000EE91FF1FA890FF1F6A91FF1F28BD0000C9
:1076D00030C80110880040006B91FF1FC020074098
:1076E0009490FF1FEC90FF1F4091FF1F6A88A988AC
:1076F0009F4B53F8084CA3F10C00BCB133F80C6C51
:10770000964209D133F80A6C8E4205D1120A032A37
:107710000CBF2378038911E00C33EAE7954A11681E
:10772000954A1160A978954A117004E0944B0F2294
:107730001A7027E000231C4600E00223EE88B342C3
:1077400038BF1E46402E34BF3546402520462946C8
:10775000FFF77CFD761B2C4403D1402D12D135461A
:1077600003E0402E34BF3546402520462946FFF72A
:107770006DFD761B2C4401D1402D03D1814AC8F800
:10778000004016800122804B3DE0804B1A8842F277
:1077900021039A4210D100237D4AC85C98540133DA
:1077A000072BF9D11368862B02D17A4B0F221A705E
:1077B00000200146FFF74AFD774B44F8383023E0BC
:1077C000764E3568B5B1DFF8BC81B8F80090B9F1F4
:1077D000400F34BF4C46402428462146FFF736FD73
:1077E000C4EB09039BB2A8F800300BB9402C00D1C0
:1077F0002B193360654B1A88B2F5A06F04D10022B3
:107800005A709A78664B1A7001225F4B6CE004EB59
:10781000C806013D736802F00802A3F10800EDB24A
:1078200002F0FF01002A36D000F036F95D485E4BC9
:1078300050F82520EAB1516840F8251002F10801FE
:107840007160595D03290BD8DFE801F002040608D6
:10785000032104E0022102E0052100E00421595542
:1078600016F0080F12880CBF8823C82343EA02438E
:1078700042E05A5D032A07D8DFE802F040400204E4
:10788000002206E0012204E016F0080F0CBF0222DD
:1078900003225A5532E054F83820120C23F8082CF1
:1078A00022B3DFF834E123F8061C43F8041C5EF829
:1078B00025303E4913B94EF8250002E051F8253035
:1078C00058603B4B41F8250033F815100A4423F863
:1078D000152000F0C3F810B10830706006E0354B99
:1078E00044F838001A7801321A7007E02A4B324AFD
:1078F00016F0080F08BF134644F8383008233B70D1
:1079000070E5E0071FD520492B482C4C02230B7053
:107910002B4B1A702B4B186098602B48D8601A615B
:107920009A615C60164B0D2018702848FF23037085
:107930002B700274264A1370264B9F221A70012363
:107940000B70BDE8F88F210604D50D4B0D221A707F
:1079500080232B70A20705D51C4B1A78D2B21A705F
:1079600002232B70E30644BF10232B70BDE8F88F71
:1079700038BD0000D489FF1F0092FF1F8491FF1FB4
:10798000C02007406891FF1F942007406091FF1FAF
:10799000F891FF1FFD90FF1FC80040009490FF1F4B
:1079A000982007404091FF1FA890FF1F9890FF1F4D
:1079B000EE91FF1F6A91FF1F88004000AC90FF1FEF
:1079C000FC90FF1F0080FF1F0091FF1F88200740D1
:1079D0008C20074084200740EC90FF1F08B500F082
:1079E00053FD00221A4B0021D15098180832882AE2
:1079F0004160F7D1174A106840F48020106002F50A
:107A000028326832C3F307201070C3F307401B0EFF
:107A100010751376FF2302F81C3C02F8143C02F8A0
:107A20008C3C012302F8083C82F8641002F8183CF0
:107A3000094B70226FF450711A700B444FF40072AE
:107A40001A6003F1C04303F5C82310221A7008BD61
:107A50000080FF1F3480044049E400E072B60C4A05
:107A60001168B1FA81F30B2B02D962B6002070477E
:107A70004FF00040D84021EA0001116062B605498C
:107A800048225343C8180022CA504260704700BFC2
:107A90007487FF1F0084FF1F0C4B4822C31AB3FBDF
:107AA000F2F30B2B11D80A4A127822B1094A127844
:107AB0000AB1FFF719BC72B6074A4FF0004121FA2C
:107AC00003F311681943116062B670470084FF1F09
:107AD0006A91FF1F7391FF1F7487FF1F10B5104C31
:107AE00023686BB120684288531C0244147A0288D0
:107AF000934212D3FFF7D0FF094B00221A600DE02A
:107B0000084B1B7813B94FF0FF3010BD0320FFF76F
:107B1000BDFB20600028E5D1F5E74380204610BD7D
:107B20008091FF1F7391FF1F10B50B4C236813B199
:107B300023686BB902E0094B1B7813B94FF0FF3093
:107B400010BD0320FFF7A2FB20600028F0D1F5E76D
:107B50005A881344187A10BD8091FF1F7391FF1F3C
:107B6000044B9888044B1B681BB11A885B88D31A96
:107B700018447047EE91FF1F8091FF1F2DE9F843D5
:107B80002D4E012307460C463370002C4FD02B4D51
:107B90002B68A9462BBB4AF2F928294B1B7803F026
:107BA000FF020BB9327015E00420FFF78BFB0728AA
:107BB00008D801233370FFF751FFC9F8000080B9DE
:107BC0001D4B1870B8F101081E4B01D01A782AB16C
:107BD00001221A704FF0FF30BDE8F88300F016FC68
:107BE000DBE72968174A488800231370C0F1400278
:107BF000944238BF224600F1080C10448C4448805F
:107C0000A41A934204D0F85C0CF803000133F8E79F
:107C10001F444B883F2B06D940230B800420FFF7DD
:107C20009FFB00232B60084B05221A70ADE73470D0
:107C30002046BDE8F88300BF7691FF1F7891FF1FB3
:107C40007391FF1F7C91FF1F7591FF1F07B502AB5A
:107C5000012103F8010D1846FFF790FF03B05DF80E
:107C600004FBFFFF2DE9F041114B1B78F3B1114EDE
:107C7000114B3468114D01271F7098464CB10027F5
:107C800063882F70042023802146FFF769FB37604B
:107C900009E0FFF7E3FE014620B104202C70FFF756
:107CA0005FFB00E02F70002388F80030BDE8F08112
:107CB0007391FF1F7891FF1F7691FF1F7591FF1F32
:107CC00038B50E4B1B7803F0FF05ABB90C4C21689F
:107CD00031B14B880B800420FFF742FB256038BD93
:107CE000FFF7BCFE014620B10420BDE83840FFF795
:107CF00037BB044B01221A7038BD00BF7691FF1FBD
:107D00007891FF1F7591FF1F08B50368C9B21B6802
:107D1000984708BD08B50368C9B21B68984708BDF5
:107D200008B50368C9B21B68984708BD08B5036861
:107D3000C9B21B68984708BD4B0803F1376000F5CE
:107D4000D830B0FBF1F0FEF733BA10B54B0803F1B1
:107D5000376000F5D8301446B0FBF1F0FEF728FA92
:107D60002046BDE81040FEF769BAFEF791BA084612
:107D7000FEF7C2BA08B50846FEF7DAFA003018BFB7
:107D8000012008BD08B50846FEF7F4FA003018BF18
:107D9000012008BDFEF7D8BBFEF712BCFEF7E4BB1E
:107DA000FEF7B6BBFEF726BCFEF7BCBB08B508461F
:107DB000FEF706FB012008BD08B50846FEF700FBEC
:107DC000012008BD10B5084614461146FEF742FBD7
:107DD000204610BD38B508460D4601F016F8044699
:107DE00021462846FEF736FB204638BD7047FFFF88
:107DF000044B00221A714FF47A711A73024A996087
:107E00001A6070478891FF1F00BC000008B5036826
:107E1000C9B21B68984708BD08B50368C9B21B689A
:107E2000984708BD08B50368C9B21B68984708BDE4
:107E300008B50368C9B21B68984708BD4B0803F131
:107E4000376000F5D830B0FBF1F0FEF789BC10B513
:107E50004B0803F1376000F5D8301446B0FBF1F061
:107E6000FEF77EFC2046BDE81040FEF7C7BCFEF7DB
:107E7000EFBC0846FEF720BD08B50846FEF738FD02
:107E8000003018BF012008BD08B50846FEF752FDB6
:107E9000003018BF012008BDFEF736BEFEF770BEE9
:107EA000FEF742BEFEF714BEFEF784BEFEF71ABE12
:107EB00008B50846FEF75CFD012008BD08B5084678
:107EC000FEF756FD012008BD10B5084614461146C0
:107ED000FEF79CFD204610BD38B508460D4600F063
:107EE00094FF044621462846FEF790FD204638BD03
:107EF0007047FFFF044B00221A714FF47A711A7316
:107F0000024A99601A6070479891FF1F58BC0000A0
:107F100008B50368C9B21B68984708BD08B503686F
:107F2000C9B21B68984708BD08B50368C9B21B6889
:107F3000984708BD08B50368C9B21B68984708BDD3
:107F40004B0803F1B76000F55840B0FBF1F0FEF7C5
:107F5000E9BE10B54B0803F1B76000F55840144670
:107F6000B0FBF1F0FEF7DEFE2046BDE81040FEF764
:107F70001BBFFEF743BF0846FEF774BF08B50846AF
:107F8000FEF78CFF003018BF012008BD08B5084679
:107F9000FEF7A6FF003018BF012008BDFFF734B878
:107FA000FFF76EB8FFF740B8FFF712B8FFF782B8D7
:107FB000FFF718B808B50846FEF7B0FF012008BD66
:107FC00008B50846FEF7AAFF012008BD10B508460F
:107FD00014461146FEF7F0FF204610BD38B508469E
:107FE0000D4600F012FF044621462846FEF7E4FF46
:107FF000204638BD7047FFFF044B00221A714FF432
:108000007A711A73024A99601A607047A891FF1F2B
:10801000B0BC000008B5034B01221A60024B1B687C
:10802000984708BD0C710340C091FF1F08B5034B72
:1080300001221A60024B5B68984708BD1C7103401F
:10804000C091FF1F08B5034B01221A60024B9B68C9
:10805000984708BD2C710340C091FF1F08B5034B22
:1080600001221A60024BDB68984708BD3C7103404F
:10807000C091FF1F054B1A6842F400021A60044BBE
:1080800000221A60034B01221A7070473C800440A2
:1080900000700340BC91FF1F064B01221A6003F5DC
:1080A00088333C331A6822F400021A60024B002223
:1080B0001A70704700700340BC91FF1FF0B54578FF
:1080C000134C144F2B011A194260134A9E188660F4
:1080D000066947F8256000259D50195103219950E4
:1080E0004378427B4433DBB2037303F1604303F50F
:1080F000644301211A70027B53119B0003F160431A
:1081000003F5614302F01F0201FA02F21A60F0BDAA
:1081100000710340C091FF1F08710340F8B50C4B7C
:108120001B7806460F460BB9FFF7A4FF0024094D44
:10813000625DE3B23AB9304673703946FFF7BEFF6D
:1081400001202855F8BD0134042CF0D10020F8BDE1
:10815000BC91FF1FB891FF1F8268002310B5136008
:10816000027B0121541102F01F0201FA02F20849B8
:1081700041F82420074A41785354D15C31B9013386
:10818000042BFAD1BDE81040FFF786BF10BD00BF39
:1081900080E100E0B891FF1F037870B504460D46FA
:1081A00016461BB1FFF7D8FF002323702561204638
:1081B0003146FFF7B3FF10B10123237000E02070B8
:1081C000207870BD037810B504460BB1FFF7C4FFEB
:1081D0000023237010BD08B5F8F744F9F8F7ACFA9E
:1081E00000F014F9FAE700F0EFBC00F0F5BC2DE95F
:1081F000F04100258C688AB0074688462E4694B127
:108200002B46404601A9212200F0E7F83B68202CCC
:1082100034BF224620225B68384601A91544A41ABF
:1082200098470644EBE730460AB0BDE8F081FFFF0F
:1082300007B5064B1B88ADF80430036801A95B68DD
:108240000222984703B05DF804FB00BF00BD0000A8
:1082500008B503685B689847002008BD0EB403B5F5
:1082600003AA52F8041B019200F0C0FE02B05DF8B0
:1082700004EB03B0704770B505468AB022B90368B5
:10828000C9B21B6898472CE0012A08BF0A2221B90D
:1082900030228DF82520212413E02124B1FBF2F0B7
:1082A00002FB1011C9B209290AAE94BF303137312F
:1082B0002644C9B206F8241C014610B1013CE4B2C0
:1082C000ECE733B1013CE4B20AAB23442D2203F8BE
:1082D000242C2B6801A95B6828462144C4F12202A2
:1082E00098470AB070BD0029BABF49422D23002328
:1082F0000A22FFF7C0BFFFF733BCFFF7EFBBFFF762
:1083000013BCFFF7AFBC0846FFF7A0BC08461146F8
:10831000FFF734BC7047FFFF044B00221A714FF483
:108320007A711A73024A99601A607047D091FF1FE0
:1083300010BD000010B50446006800F04DFC20465A
:1083400010BD38B504460D460068013100F024FD2B
:1083500010B184E82100012038BD43688B4210B57C
:10836000044606D2FFF7EDFF20B1A3680BB92268DF
:108370001370012010BDF8B504460F46154622B90A
:10838000036803B11A7000230BE01146FFF7E5FF05
:10839000064640B9206810B100F01EFC266000239C
:1083A0006360A36004E0A5602068394600F025FD05
:1083B0002046F8BD38B5002304460360436083605F
:1083C00003730D4639B1084600F01FFD29460246E9
:1083D0002046FFF7D0FF204638BD38B50C469AB18D
:1083E00091B181688B4202D30023237038BDC91A32
:1083F000551E8D4228BF0D4601682A461944204665
:1084000000F022FD0023635538BDFFFF10B50E4C70
:108410002378BBB901232370FFF7A2FB08B1FFF754
:1084200079FFFEF791F808B1FFF7E0FCFEF76CFB6F
:1084300008B1FFF75DFDFEF7E7FD08B1FFF7DAFDD4
:108440000023237010BD00BFE091FF1F10B5002373
:10845000B0FBF2F402FB1400092894BF303037302F
:10846000C0B2C85420460CB10133F1E7CA185470A9
:1084700022469A4206DA885CCC5C8C54C85401329D
:10848000013BF6E7084610BD1FB572B6154B7022CA
:108490001A70154A412111700F2102F8011C802227
:1084A0001A701A781206FCD5104B186862B6104B79
:1084B000984298BF0A2301AC98BF584321460A222C
:1084C000FFF7C4FF0023E15C0A4A29B102EB430035
:1084D00001330A2B4180F6D101335B00137004B0E5
:1084E00010BD00BF0000024007000240080002402B
:1084F0007F9698000088FF1F80F0004002E000BFD8
:1085000081F0004142001FBF5FEA410392EA030F7E
:108510007FEA226C7FEA236C6AD04FEA1262D2EBC8
:108520001363C1BFD218414048404140B8BF5B42CD
:10853000192B88BF704710F0004F40F4000020F066
:108540007F4018BF404211F0004F41F4000121F07C
:108550007F4118BF494292EA030F3FD0A2F10102C6
:1085600041FA03FC10EB0C00C3F1200301FA03F104
:1085700000F0004302D5494260EB4000B0F5000F27
:1085800013D3B0F1807F06D340084FEA310102F1E6
:108590000102FE2A51D2B1F1004F40EBC25008BF98
:1085A00020F0010040EA03007047490040EB000062
:1085B00010F4000FA2F10102EDD1B0FA80FCACF191
:1085C000080CB2EB0C0200FA0CF0AABF00EBC25090
:1085D00052421843BCBFD0401843704792F0000F7E
:1085E00081F4000106BF80F400000132013BB5E7D1
:1085F0004FEA41037FEA226C18BF7FEA236C21D047
:1086000092EA030F04D092F0000F08BF08467047AB
:1086100090EA010F1CBF0020704712F07F4F04D179
:10862000400028BF40F00040704712F100723CBF8C
:1086300000F50000704700F0004343F0FE4040F4B6
:10864000000070477FEA226216BF08467FEA236374
:108650000146420206BF5FEA412390EA010F40F45F
:10866000800070474FF0000304E000BF10F00043AB
:1086700048BF40425FEA000C08BF704743F0964392
:1086800001464FF000001CE050EA010208BF7047AD
:108690004FF000030AE000BF50EA010208BF704734
:1086A00011F0004302D5404261EB41015FEA010C49
:1086B00002BF84460146002043F0B64308BFA3F141
:1086C0008053A3F50003BCFA8CF2083AA3EBC25323
:1086D00010DB01FA02FC634400FA02FCC2F1200242
:1086E000BCF1004F20FA02F243EB020008BF20F079
:1086F0000100704702F1200201FA02FCC2F12002DF
:1087000050EA4C0021FA02F243EB020008BF20EAD3
:10871000DC7070474FF0FF0C1CEAD0521EBF1CEA01
:10872000D15392EA0C0F93EA0C0F6FD01A4480EAEF
:10873000010C400218BF5FEA41211ED04FF00063D8
:1087400043EA501043EA5111A0FB01310CF0004004
:10875000B1F5000F3EBF490041EAD3715B0040EA2A
:10876000010062F17F02FD2A1DD8B3F1004F40EBFA
:10877000C25008BF20F00100704790F0000F0CF0CD
:10878000004C08BF49024CEA502040EA51207F3A91
:10879000C2BFD2F1FF0340EAC250704740F400006C
:1087A0004FF00003013A5DDC12F1190FDCBF00F05D
:1087B00000407047C2F10002410021FA02F1C2F10B
:1087C000200200FA02FC5FEA310040F1000053EAA7
:1087D0004C0308BF20EADC70704792F0000F00F0F5
:1087E000004C02BF400010F4000F013AF9D040EAFB
:1087F0000C0093F0000F01F0004C02BF490011F48F
:10880000000F013BF9D041EA0C018FE70CEAD1538C
:1088100092EA0C0F18BF93EA0C0F0AD030F0004C0C
:1088200018BF31F0004CD8D180EA010000F00040C0
:10883000704790F0000F17BF90F0004F084691F07E
:10884000000F91F0004F14D092EA0C0F01D14202B8
:108850000FD193EA0C0F03D14B0218BF084608D181
:1088600080EA010000F0004040F0FE4040F40000CB
:10887000704740F0FE4040F4400070474FF0FF0C5E
:108880001CEAD0521EBF1CEAD15392EA0C0F93EAA5
:108890000C0F69D0A2EB030280EA010C49024FEAF7
:1088A000402037D04FF0805343EA111143EA1013B0
:1088B0000CF000408B4238BF5B0042F17D024FF468
:1088C000000C8B4224BF5B1A40EA0C00B3EB510F43
:1088D00024BFA3EB510340EA5C00B3EB910F24BF2C
:1088E000A3EB910340EA9C00B3EBD10F24BFA3EBB1
:1088F000D10340EADC001B0118BF5FEA1C1CE0D179
:10890000FD2A3FF650AF8B4240EBC25008BF20F02B
:10891000010070470CF0004C4CEA50207F32C2BF7F
:10892000D2F1FF0340EAC250704740F400004FF01C
:108930000003013A37E792F0000F00F0004C02BF4D
:10894000400010F4000F013AF9D040EA0C0093F017
:10895000000F01F0004C02BF490011F4000F013B71
:10896000F9D041EA0C0195E70CEAD15392EA0C0FD9
:1089700008D142027FF47DAF93EA0C0F7FF470AF11
:10898000084676E793EA0C0F04D14B023FF44CAF54
:1089900008466EE730F0004C18BF31F0004CCAD1E9
:1089A00030F000427FF45CAF31F000437FF43CAF25
:1089B0005FE700BF4FF0FF3C06E000BF4FF0010C47
:1089C00002E000BF4FF0010C4DF804CD4FEA400229
:1089D0004FEA41037FEA226C18BF7FEA236C11D073
:1089E00001B052EA530C18BF90EA010F58BFB2EB26
:1089F000030088BFC81738BF6FEAE17018BF40F0A6
:108A0000010070477FEA226C02D15FEA402C05D159
:108A10007FEA236CE4D15FEA412CE1D05DF8040BDE
:108A2000704700BF844608466146FFE70FB5FFF771
:108A3000C9FF002848BF10F1000F0FBD4DF808ED29
:108A4000FFF7F4FF0CBF012000205DF808FB00BF1A
:108A50004DF808EDFFF7EAFF34BF012000205DF874
:108A600008FB00BF4DF808EDFFF7E0FF94BF0120C1
:108A700000205DF808FB00BF4DF808EDFFF7D2FFBE
:108A800094BF012000205DF808FB00BF4DF808ED01
:108A9000FFF7C8FF34BF012000205DF808FB00BFCE
:108AA0004FEA4002B2F1FE4F0FD34FF09E03B3EBFB
:108AB00012620DD94FEA002343F0004310F0004F3B
:108AC00023FA02F018BF404270474FF00000704791
:108AD00012F1610F01D1420205D110F0004008BF30
:108AE0006FF0004070474FF00000704742000ED218
:108AF000B2F1FE4F0BD34FF09E03B3EB126209D4D9
:108B00004FEA002343F0004323FA02F070474FF08E
:108B10000000704712F1610F01D1420202D14FF003
:108B2000FF3070474FF00000704700BF0346084613
:108B3000194600F013B800210A2200F019BA0021EA
:108B40000A2200F015BAFFFF0A46034903460868E7
:108B5000194600F07BB800BF7888FF1F70B5064C3F
:108B600006460D4613462CB131462A460220AFF385
:108B7000008070BD204670BD0000000070B50E4B37
:108B80000E4DED1AAD1000241E46AC4204D056F82E
:108B9000242090470134F8E703F0C2F9084D094B4F
:108BA000ED1AAD1000241E46AC4204D056F8242025
:108BB00090470134F8E770BD2CBF00002CBF0000C7
:108BC00044BF00002CBF0000024B0146186800F0B3
:108BD0008FB800BF7888FF1F024B0146186800F06D
:108BE00043B800BF7888FF1F10B5C9B20244904255
:108BF000034606D01C788C4200F10100F7D11846DC
:108C000010BD002010BD814270B501D300230EE0DD
:108C10008C18A042FAD28518134613F1FF3305D3FE
:108C2000514266182944F65CCE54F6E770BD934273
:108C300003D0CC5CC4540133F9E770BD0244034651
:108C4000934202D003F8011BFAE7704738B502FBE4
:108C500001F4214600F04CF8054618B100212246E7
:108C6000FFF7ECFF284638BD30B500293CD051F85D
:108C7000042C0B1F1D49002AB8BF9B180A680C461C
:108C800012B95A600B6030BD93420DD21968581862
:108C9000904203D15A581144426819605A602360C7
:108CA00030BD994203D80A4651680029F9D11468A9
:108CB00015199D420AD11B682344D01888421360BD
:108CC00012D10868034413604B680CE002D90C23EE
:108CD000036030BD18681C188C4203D10C684968C9
:108CE000204418605960536030BD00BFE891FF1FF9
:108CF00070B5CD1C25F0030508350C2D38BF0C25AB
:108D0000002D06463FDB8D423DD3214B1C681846A3
:108D10002146A1B10B685B1B0ED40B2B03D90B6052
:108D2000CC18CD501FE08C4202D1626802601AE07C
:108D30004B6863600C4616E00C464968E9E7154C41
:108D400023681BB9304600F031F8206029463046D0
:108D500000F02CF8431C014615D0C41C24F0030479
:108D600084420AD1256004F10B00231D20F0070086
:108D7000C31A0BD05A42E25070BD3046611A00F05F
:108D800015F80130EED10C233360002070BD00BF18
:108D9000E891FF1FE491FF1F0A4603490346086854
:108DA000194600F001BA00BF7888FF1F38B5064C9D
:108DB0000023054608462360FCF71EFE431C02D133
:108DC000236803B12B6038BD0492FF1FC9B202466D
:108DD00010F8013B1BB18B42F9D1104670470029B6
:108DE000FBD01846704710F8012B11F8013B012AFF
:108DF00028BF9A42F7D0D01A7047034611F8012BCA
:108E000003F8012B002AF9D17047034613F8012B10
:108E1000002AFBD1181A0138704770B592B10B4681
:108E200005461C7810F8016BB44201F1010101D133
:108E3000012A03D128781B78C01A70BD013A002C92
:108E4000EDD1F7E7104670BD10B5034632B111F809
:108E5000014B03F8014B013A002CF7D11A4493421D
:108E600003D0002103F8011BF9E710BD84463F48F9
:108E70002DE9F04FD0F800800E46344614F8015B1F
:108E800008EB0500407800F0080000F0FF0708B18B
:108E90002646F2E72D2D03D1B41C7578012703E097
:108EA0002B2D04BF7578B41C33F010000DD1302D7C
:108EB00008D1207800F0DF00582851D165781023C0
:108EC000023402E0002B08BF0A23002F0CBF6FF012
:108ED000004A4FF0004ABAFBF3F9002603FB19AA37
:108EE000304608EB050B9BF801B01BF0040F01D0D6
:108EF000303D0BE01BF0030B1BD0BBF1010F14BF87
:108F00004FF0570B4FF0370BCBEB05059D4210DAB6
:108F1000B6F1FF3F0AD0484506D801D1554503DCDC
:108F200003FB0050012601E04FF0FF3614F8015B0F
:108F3000D7E7731C0CD1002F4FF022030CBF6FF04A
:108F400000404FF00040CCF800302AB9BDE8F08F67
:108F500007B1404242B106B1611E1160BDE8F08F19
:108F6000002B08BF0823B0E7BDE8F08F7C88FF1F07
:108F700030B51346044A05460C4610682946224679
:108F8000BDE83040FFF772BF7888FF1F2DE9F04140
:108F9000ADF5047D1D464FF400730F4690460393D4
:108FA000044618B183690BB900F094F804AE00953B
:108FB0002046314603AA434600F05FF9054670B1EA
:108FC000204639462A46039B00F01EF8B54203901E
:108FD00003D020462946FFF747FE039801E04FF0F3
:108FE000FF300DF5047DBDE8F081FFFF30B513467D
:108FF000044A05460C46106829462246BDE8304022
:10900000FFF7C4BF7888FF1F38B5074C054600201E
:109010002060084611461A46FFF71AF9431C02D190
:10902000236803B12B6038BD0492FF1FF8B50746D3
:1090300000F1480494B1A5686668013E0CD4AB8980
:10904000012B07D9B5F90E30013303D03846294634
:1090500000F0D6F96835F0E72468EBE7F8BDFFFFCC
:10906000002310B50446036043608360818143663A
:10907000C28103614361836119465C300822FFF7B6
:10908000DDFD054B6362054BA362054BE362054BB7
:109090002462236310BD00BFF59100001792000009
:1090A0004F9200007392000070B54B1E68255D431F
:1090B0000E4605F17401FFF71BFE044640B1002186
:1090C00080E842000C30A06005F16802FFF7B6FDB1
:1090D000204670BD836910B5044633BB8364C36406
:1090E0000365124B124A1B688262984204BF012337
:1090F000836100F01FF86060204600F01BF8A0605C
:10910000204600F017F80421E06000226068FFF7B5
:10911000A7FFA06809210122FFF7A2FFE068122142
:109120000222FFF79DFF0123A36110BD84BD000053
:109130002D900000F8B51B4B1E68B369074613B9A4
:109140003046FFF7C7FF4836B4687368013B04D464
:10915000B4F90C5075B16834F8E733682BB9384668
:109160000421FFF7A1FF306008B13668ECE70C235B
:109170003B60F8BD4FF6FF73E3810123A381656671
:109180002560A560656025616561A56104F15C00ED
:1091900029460822FFF752FD6563A563A564E564CF
:1091A0002046F8BD84BD0000F8B5064614460D46BD
:1091B00021B91146BDE8F840FFF79ABD1AB9FFF78B
:1091C00053FD2046F8BD00F057F9A0420ED23046BC
:1091D0002146FFF78DFD074650B129462246FCF790
:1091E00053F830462946FFF73FFD01E02846F8BD19
:1091F0003846F8BD10B50C46B1F90E1000F046F92E
:10920000002803DB636D0344636510BDA38923F469
:109210008053A38110BD2DE9F0411D468B89DB05EC
:1092200007460C46164605D5B1F90E10002202235A
:1092300000F010F9A389B4F90E1023F48053A38130
:10924000384632462B46BDE8F041FFF7DDBE10B58B
:109250000C46B1F90E1000F0FDF8431CA38903D1B0
:1092600023F48053A38110BD43F48053A381606530
:1092700010BDB1F90E1000F02FB830B515469BB0F7
:10928000146829B124B14FF4C162ADF80C2005E097
:109290004FF422720024ADF80C202146002C0091DE
:1092A000049103DA8B230360002012E04FF6FF7273
:1092B000ADF80E2069461A461E9B0294059400F0F4
:1092C00053F9031E4FF0000003DB2B60009B187066
:1092D00004981BB030BDFFFF38B5064C002305468F
:1092E00008462360FCF792FB431C02D1236803B1BC
:1092F0002B6038BD0492FF1F8A892DE9F041054695
:1093000010070C4657D44B68002B02DC0B6C002B6B
:1093100018DDE66AB6B102F48052002392B22F68DB
:109320002B600AB1626D10E0216A28460123B04724
:10933000411C024609D12B683BB11D2B01D0162BD5
:1093400046D12F600020BDE8F081A3895B0705D5D9
:109350006368D21A636B0BB1236CD21AE66A216A76
:1093600028460023B047461CA28905D12B681BB1B3
:109370001D2B01D0162B19D100236360D104236962
:10938000236004D5421C01D12B6803B96065616B71
:109390002F600029D6D004F14403994202D0284618
:1093A000FFF762FC00206063BDE8F08142F04002FC
:1093B000A281BDE8F0810E69002EC3D00B680E605B
:1093C000C6EB030893070CBF4B6900238B6012E0C8
:1093D000A38943F04003A3814FF0FF30BDE8F08143
:1093E000A76A216A284632464346B8470028EFDD7F
:1093F0000644C0EB0808B8F1000FF1DCA2E7FFFF5C
:1094000038B50B6905460C46DBB118B183690BB959
:10941000FFF760FE0C4B9C4201D16C6808E00B4BDF
:109420009C4201D1AC6803E0094B9C4208BFEC6848
:10943000B4F90C302BB128462146BDE83840FFF77F
:109440005BBF002038BD00BF8CBE0000ACBE00007A
:10945000CCBE000038B5074C054600202060084609
:1094600011461A46FCF7D5FA431C02D1236803B112
:109470002B6038BD0492FF1F51F8040C002802DA5B
:1094800004390B58184404387047FFFF38B5074CAF
:10949000054600202060084611461A46FCF7B4FA3B
:1094A000431C02D1236803B12B6038BD0492FF1F17
:1094B0002DE9F0478D68AB4281460C4692461F4627
:1094C00043D38B8913F4906F3DD026680969C1EBB3
:1094D00006086669022206EB460696FBF2F608F1DC
:1094E00001023A44964238BF16465B050FD5314615
:1094F000FFF7FEFB054698B121694246FBF7C4FE23
:10950000A38923F4906343F08003A38113E03246E0
:10951000FFF74AFE054670B948462169FFF7A4FBEC
:109520000C23C9F80030A38943F04003A3814FF016
:10953000FF30BDE8F087256166614544C8EB06064B
:109540002560A6603D46AF4200D23D462A462068CF
:109550005146FFF758FBA3685B1BA36023681D44BB
:1095600025600020BDE8F0872DE9F0439DB0074657
:1095700003938B891C060D4616460CD50B6953B90F
:109580004021FFF7B5FB2860286110B90C233B6030
:10959000C8E040236B610023099320238DF8293014
:1095A00030238DF82A3033461C4613F8012B1AB9A4
:1095B000B4EB06090FD002E0252AF5D1F8E73846CA
:1095C000294632464B46FFF773FF013000F0A58075
:1095D000099B4B4409932378002B00F09E800023C5
:1095E0004FF0FF3204930793059206938DF85330A2
:1095F0001A9304F101094C464D4E2178304605225C
:10960000FFF7F2FA09F10109049B28B1861B01203A
:10961000B04003430493EEE7D90644BF20228DF8FF
:1096200053201A0744BF2B228DF8532022782A2A70
:1096300002D0079B21460EE0039A111D1268039188
:10964000002A01DB079204E0524243F00203079232
:10965000049301340AE00C4601312278303A092A99
:1096600003D80A2000FB0323F5E7079323782E2B6A
:109670001AD163782A2B0AD1039B1A1D1B68039207
:10968000002B04F10204B8BF4FF0FF330BE0611C64
:1096900000230C4601312278303A092A03D80A20E7
:1096A00000FB0323F5E70593224E21783046032281
:1096B000FFF79AFA30B1861B049B4020B040034369
:1096C0000493013421781C488DF828100622661C6A
:1096D000FFF78AFA88B1194B33B9039B073323F09C
:1096E00007030833039314E003AB0093384604A93F
:1096F0002A46134BAFF3008007E003AB00933846D4
:1097000004A92A460E4B00F08FF8B0F1FF3F8046C7
:1097100003D0099B4344099345E7AB895B0601D419
:10972000099801E04FF0FF301DB0BDE8F08300BFA5
:10973000ECBE0000F2BE0000F6BE0000000000001B
:10974000B19400002DE9F84315461F468A680B695D
:10975000DDF820809A42A8BF13462B6091F8432081
:1097600006460C460AB101332B602368990602D5E0
:109770002B6802332B60236813F006091DD094F880
:1097800043302268003318BF012392061FD5E11829
:109790005A1C302081F84300224494F8451082F886
:1097A0004310023313E03046394604F11902012315
:1097B000C047013007D009F10109E2682B68D31ACC
:1097C0009945F0DBDBE74FF0FF30BDE8F88330462A
:1097D000394604F14302C0470130F4D023682A68B7
:1097E000E16803F00603042B08BFC2EB01052369FF
:1097F000A2680CBF25EAE57500259A42C4BFC3EBF9
:109800000203ED184FF00009A9450ADA304639463F
:1098100004F11A020123C0470130D4D009F1010933
:10982000F2E70020BDE8F8832DE9FF470E7E0C9D8E
:109830006E2E80460C4691469A4601F1430000F098
:10984000A58011D8632E22D009D8002E00F0AF8059
:10985000582E40F0BF8081F845607B4A4FE0642E6F
:109860001ED0692E1CD0B5E0732E00F0A48009D85C
:109870006F2E2BD0702E40F0AD800B6843F020038C
:109880000B6038E0752E21D0782E34D0A2E02B6802
:109890001A1D1B682A6001F1420781F842309DE0E1
:1098A00022682B6812F0800F03D01A1D2A601D68F1
:1098B00005E05106F9D51A1D2A60B3F90050002DB4
:1098C00039DA2D236D4284F8433034E022682B6866
:1098D00012F0800F03D01A1D2A601D6804E05206A2
:1098E000F9D51A1D2A601D88237E574A6F2B14BF95
:1098F0000A2308231BE07823544A84F84530236860
:10990000296813F0800F01F104062E6001D00D6864
:1099100002E05F06FBD50D88DE0744BF43F020035D
:1099200023601DB9236823F0200323601023002146
:1099300084F8431001E0444A0A236668A660002EBA
:1099400003DB216821F00401216005B96EB104F147
:109950004201B5FBF3F603FB16550F46555D01F8C2
:1099600001593546002EF4D100E00746082B0AD1F4
:109970002368DD0707D5626823699A4203DC302338
:1099800007F8013C013FC01B20612CE009682B68EF
:10999000626911F0800F04D0191D29601B681A60DC
:1099A00005E04906F8D5191D29601B681A800023B7
:1099B0002361074617E02B681A1D2A601F68384686
:1099C000FFF723FA63682061984288BF2361236907
:1099D000636005E004F1420784F8426001232361DB
:1099E000002384F84330CDF800A04046214603AA66
:1099F0004B46FFF7A7FE013002D14FF0FF301FE0CA
:109A0000404649463A462369D0470130F5D023689D
:109A10009B0705D4E068039B9842B8BF18460FE047
:109A20000025E268039BD31A9D42F3DA404649467B
:109A300004F119020123D0470130DED00135F0E7EF
:109A400004B0BDE8F08700BFFDBE00000EBF0000FF
:109A5000436F6E6E656374656420746F2045524F6A
:109A60005320626F61726420617420256462707398
:109A70002E20426F617264204657207665727369AA
:109A80006F6E2025642E0A0A427269646765206D34
:109A90006F646520656E61626C656420666F72201C
:109AA000496E7465726E616C2044657669636520E9
:109AB000626F6F746C6F616465722061636365735C
:109AC000732E0A57616974696E6720666F7220741D
:109AD000686520666972737420636861726163747B
:109AE000657220746F2072657365742074686520D8
:109AF000696E7465726E616C205053552E2E2E2E39
:109B0000005B4254204E4F542050524553454E5412
:109B10005D0041542B554152543D25642C302C306E
:109B2000000D0A004F4B0041540041542B4E414D53
:109B3000453F0041542B505357443F005B4D414932
:109B40004E4252445F554E535550525445445D0069
:109B500041542B4E414D453D25730041542B5053EC
:109B600057443D2530346900636C735F4369726309
:109B70004275666665725F3100636C734369726338
:109B80004275666665725F320044756D70696E6716
:109B90002043697263756C617220627566666572D6
:109BA0005F006275666665725F2073697A65206919
:109BB000733A2025640A00252E32782000FFFFFF2B
:109BC0000000000000000000195A00000915000004
:109BD00021150000000000001801FFFFFFFFFFFF3C
:109BE00000000000000000004915000015150000ED
:109BF00035150000000000005B74696D656F7574B9
:109C00005D0A005B25645D205B25645D0A005B7076
:109C10006172616D735F636F756E742025645D2082
:109C20005B25645D0A00556E6B6E6F776E207374F2
:109C300061746520696E2063616C6C6261636B2086
:109C4000696E20636C73436F6E736F6C65212121A5
:109C50000A00496E69742064796E207061636B65D7
:109C6000740050617274696C6C79206F70656E203D
:109C700068616E642066756E6374696F6E616C698D
:109C80007479206973206E6F742079657420696D12
:109C9000706C656D656E74656420696E20746869AA
:109CA00073206669726D776172652076657273697B
:109CB0006F6E2E20504C656173652075736520743E
:109CC000686520636F6D6D616E6420746F207365CD
:109CD0007420736572766F20706F736974696F6E2C
:109CE0007320696E646976696475616C6C792E0A9B
:109CF00000436C6F73652068616E642066756E63E7
:109D000074696F6E616C697479206973206E6F7409
:109D10002079657420696D706C656D656E7465641D
:109D200020696E20746869732076657273696F6E3E
:109D30002E205573652074686520636F6D6D616EAC
:109D40006420746F2073657420736572766F207061
:109D50006F736974696F6E7320696E646976696484
:109D600075616C6C792E0A005363616E6E696E6763
:109D700020696E2070726F677265732E205573654F
:109D800020636F6D6D616E642027737461747573E9
:109D90002720746F206C6973742049447320666FA8
:109DA000756E642E00596573004E6F0053656564CF
:109DB00020526F626F746963732045524F5320467F
:109DC00069726D776172650A00426F617264206D1D
:109DD0006F64656C2025640A00426F6172642048DC
:109DE0005720436F6E66696775726174696F6E2084
:109DF00025640A004669726D776172652076657226
:109E000073696F6E2025640A0053657269616C2066
:109E10004E756D62657220252E3278252E3278259A
:109E20002E32780A0043757272656E742073656E07
:109E3000736F72207265736973746F722076616CD0
:109E400075653A2025640A00426F61726420697367
:109E500020636F6E6669677572656420746F206F2A
:109E60007065726174652077697468203132626947
:109E700074207265736F6C7574696F6E2E0A004280
:109E80006F61726420697320636F6E6669677572B3
:109E9000656420746F206F706572617465207769E6
:109EA0007468203130626974207265736F6C7574E8
:109EB000696F6E2E0A000A45787465726E616C20B7
:109EC00062757320636F6D6D756E69636174696F20
:109ED0006E2073657474696E67733A200A00426F6E
:109EE00061726420627573206465766963652049D8
:109EF000443A2025640A0052657475726E206465C8
:109F00006C61792074696D653A202564205B256455
:109F1000206D6963726F736563735D0A00537461CA
:109F20007475732072657475726E206C6576656CDD
:109F30003A2025640A005573696E672054582045FD
:109F40006E61626C652070696E3A2025730A000AA2
:109F5000496E7465726E616C2062757320636F6DFB
:109F60006D756E69636174696F6E20736574746971
:109F70006E67733A20000A496E7465726E616C20D8
:109F80006275732042617564207261746520736527
:109F90007474696E673A202564203D202564204250
:109FA00050530A000A4120426C7565746F6F7468E3
:109FB00020636F6D6D756E69636174696F6E206D7E
:109FC0006F64756C652069732070726573656E745B
:109FD0003A0A00426C7565746F6F746820434F4D88
:109FE0004D20426175642073657474696E67202525
:109FF00064203D202564204250530A00426C756560
:10A00000746F6F746820646576696365206E616D36
:10A01000653A202573200A00426C7565746F6F7471
:10A02000682064657669636520636F64653A2025FE
:10A03000303464200A000A4E6F20426C7565746FDC
:10A040006F746820636F6D6D756E69636174696F9D
:10A050006E206D6F64756C652064657465637465EE
:10A06000642E0A004F6E004F666600426F61726494
:10A07000205374617475733A0A00496E7465726E88
:10A08000616C2054656D70657261747572653A0912
:10A09000256420646567430A0045787465726E61C3
:10A0A0006C20537570706C7920566F6C74616765A5
:10A0B0003A0925642E2564560A00436F6E66696767
:10A0C0007572656420566F6C7461676520696E20D7
:10A0D000496E7465726E616C204275733A0925642D
:10A0E000560A0A00506F736974696F6E2053656E6B
:10A0F000736F722057416464756374696F6E3A09B7
:10A1000025640A00506F736974696F6E2053656E21
:10A11000736F722057466C6578696F6E3A092564D3
:10A120000A0050616C6D204F70746963616C20533C
:10A13000656E736F7220696E7374616C6C65643ADE
:10A140000925730A0050616C6D204F70746963615A
:10A150006C2053656E736F7220416D6269656E7419
:10A16000204C696768743A0925640A0050616C6D77
:10A17000204F70746963616C2053656E736F722039
:10A18000436F6D70757465642052656164696E67B4
:10A190003A0925640A0043617061636974697665F0
:10A1A0002053656E736F727320696E7374616C6C8B
:10A1B00065643A0925730A004361706163697469D3
:10A1C00076652053656E736F72203120726561640D
:10A1D000696E673A0925640A0043617061636974B6
:10A1E0006976652053656E736F72203220726561E7
:10A1F00064696E673A0925640A000A436F6D6D75DC
:10A200006E69636174696F6E2053746174697374ED
:10A210006963733A0A0055415254312028457874D5
:10A220002E436F6D6D2920427566666572204F76EC
:10A23000657272756E733A2025640A005541525456
:10A24000322028496E742E436F6D6D292042756649
:10A25000666572204F76657272756E733A2025645A
:10A260000A005541525433205B42542E436F6D6DAA
:10A270005D20427566666572204F76657272756EF6
:10A28000733A2025640A000A536572766F204944A8
:10A290007320286C6973743A2049442C205B455222
:10A2A000524F52204D41534B5D290A002564095BF2
:10A2B0004D41494E424F4152445D0A002564095BBD
:10A2C00025645D0A000A506F72742073746174759E
:10A2D000733A0A00506F72742025642043757272BD
:10A2E000656E742052656164696E673A204F564509
:10A2F000524C4F4144204552524F52202825646D04
:10A3000041290A00506F72742025642043757272CF
:10A31000656E742052656164696E673A2025646DCC
:10A32000410A000A4120426C7565746F6F746820A1
:10A33000636F6D6D756E69636174696F6E206D6FAB
:10A3400064756C652069732070726573656E742E18
:10A350000A00426C7565746F6F746820706F776562
:10A3600072207374617475733A2025730A00536503
:10A37000656420526F626F746963732045524F5356
:10A38000204669726D776172652C207665727369FB
:10A390006F6E2025640A0A004C697374206F662072
:10A3A000616476616E63656420636F6D6D616E6478
:10A3B000732E0A5741524E494E473A2054686573EE
:10A3C0006520636F6D6D616E6473206172652072CC
:10A3D0006573657276656420666F722074686520A7
:10A3E000757365206F66205365656420526F626FD8
:10A3F0007469637320746563686E6963616C20615E
:10A4000067656E74732E0A496E636F72726563744A
:10A41000207573616765206D61792063617573656F
:10A4200020696E6F7065726174696F6E2C20646153
:10A430006D61676520616E64206D617920766F695A
:10A440006420796F75722077617272616E74792EF3
:10A450000A55736520617420796F7572206F776E6D
:10A46000207269736B2E0A0A00616870095468696A
:10A4700073206D6573736167652E0A00696E697478
:10A4800020656570726F6D0A00696E697420626F75
:10A490006172646D6F64656C205B6D6F64656C5D8B
:10A4A0000A00696E697420626F6172646877636F15
:10A4B0006E666967205B636F6E666967206D6173A6
:10A4C0006B5D0A00696E69742063757272656E74E3
:10A4D0007265736973746F72205B726573697374EC
:10A4E0006F722076616C7565204F686D735D0A0030
:10A4F000696E697420736E205B59595D205B4D4D08
:10A500005D205B434845434B53554D5D0A00696EE2
:10A5100069742073657269616C636F6D6D205B6C2B
:10A520006566747C72696768745D0A0A00557365B4
:10A530002027636F6E6669672720666F72207468D4
:10A54000652072656D61696E696E6720636F6E6606
:10A55000696775726174696F6E732E2054797065C6
:10A56000202768656C702720666F7220696E666FA1
:10A57000726D6174696F6E2E0A0A004C69737420E3
:10A580006F6620617661696C61626C6520636F6DD6
:10A590006D616E64732E20416C6C20636F6D6D6114
:10A5A0006E64732061726520636173652073656EEC
:10A5B0007369746976652E0A0A0068656C700954BF
:10A5C000686973206D6573736167652E0A00737423
:10A5D0006174757309446973706C61792063757275
:10A5E00072656E742073797374656D207374617411
:10A5F00075732E0A0061626F757409446973706C1B
:10A60000617920696E7465726E616C20696E666F27
:10A61000726D6174696F6E2E0A007363616E62758C
:10A62000730952657363616E732074686520696E87
:10A630007465726E616C2062757320666F7220445F
:10A64000796E616D6978656C2064657669636573A0
:10A650002E0A00736574706F73205B64657669639E
:10A66000652069645D205B706F736974696F6E3A11
:10A6700020302D25645D0953657420706F736974F3
:10A68000696F6E20666F72207370656369666965B5
:10A6900064206465766963652E0A0072657374616F
:10A6A0007274205B7073757C616C6C5D09526573AC
:10A6B0007461727473206F6E6C7920746865207396
:10A6C0006572766F20505355206F72207468652034
:10A6D00066756C6C2073797374656D2E0A00636FF8
:10A6E0006E666967205B657874626175647C657805
:10A6F0007469647C6578747478656E61626C657C7D
:10A7000031326269746164636578706F7365647C0B
:10A71000696E74626175647C6274626175647C6286
:10A72000746E616D657C6274636F64657C62746372
:10A730006F6D6D616E645D205B76616C75655D0A41
:10A740000953797374656D207769646520636F6E52
:10A7500066696775726174696F6E206F7074696F76
:10A760006E732E0A00636F6D6D6272696467652097
:10A770005B6269746D61736B5D09456E61626C65E6
:10A7800020434F4D4D206272696467652E0A09426D
:10A7900069746D61736B3A20313D5553422C203200
:10A7A0003D496E74204275732C20343D45787420E9
:10A7B0004275732C20383D42542C2031363D555380
:10A7C0004220772F4454522052657365742E0A003C
:10A7D000777262205B6465766963652069645D20D9
:10A7E0005B616464726573735D205B62797465207C
:10A7F00076616C75655D095772697465206279745C
:10A800006520746F206465766963652E0A0077722F
:10A8100077205B6465766963652069645D205B61B0
:10A820006464726573735D205B696E742076616C1D
:10A8300075655D09577269746520776F726420745D
:10A840006F206465766963652E0A00726562205B1D
:10A850006465766963652069645D205B6164647228
:10A860006573735D09526561642062797465206661
:10A87000726F6D206465766963652E0A0072657774
:10A88000205B6465766963652069645D205B616453
:10A8900064726573735D095265616420776F7264D9
:10A8A0002066726F6D206465766963652E0A0A0002
:10A8B000496E76616C696420636F6D6D616E642EA4
:10A8C00020436F6D6D616E647320617265206361FA
:10A8D00073652073656E7369746976652E0A5479A1
:10A8E0007065202768656C702720666F72206D6F19
:10A8F000726520696E666F726D6174696F6E2E0A83
:10A90000004944206E6F742070726573656E742008
:10A91000696E2074686520696E7465726E616C2062
:10A920006275732E20547970652027737461747575
:10A93000732720666F722061206C697374206F66C4
:10A940002076616C6964204944732E0A00496E7652
:10A95000616C696420706F736974696F6E2E204D2D
:10A960006178696D756D20616363657074656420DD
:10A97000706F736974696F6E206973203430393574
:10A980002E0A41637475616C206D6178696D756D17
:10A9900020646570656E6473206F6E2061637475EA
:10A9A00061746F7220636F6E666967757261746936
:10A9B0006F6E2E0A0070737500446F6E6500616CD7
:10A9C0006C00506172616D657465722070617373A3
:10A9D00065642028222573222920697320696E76F8
:10A9E000616C69642E204269746D61736B206D75B2
:10A9F0007374207365742074776F20696E74657248
:10AA000066616365732E0A00446F6E652E0065787B
:10AA1000747478656E61626C6500796573006E6F41
:10AA20000031326269746164636578706F73656464
:10AA300000696E74626175640062746261756400BD
:10AA4000496E76616C69642073657474696E672EF3
:10AA50002053657474696E672073686F756C642029
:10AA600062652061204261756420706172616D656C
:10AA700074657220286578616D706C653A20313696
:10AA80003D31313532303062707329005375636562
:10AA9000737320636F6E6669677572696E672042B3
:10AAA00054206D6F64756C652E0A004661696C6593
:10AAB0006420636F6E6669677572696E67204254C1
:10AAC000206D6F64756C652E0A0053617665642095
:10AAD00073657474696E6720696E204D61696E20BC
:10AAE000626F61726420656570726F6D2E006274B2
:10AAF0006E616D65005375636573730A0046616925
:10AB00006C0A006274636F646500496E76616C69FB
:10AB10006420636F64652E20436F6465206D7573D8
:10AB20007420626520612034206469676974206E36
:10AB3000756D6572696320636F64652072616E670D
:10AB4000696E672066726F6D203030303020746F10
:10AB500020393939392E0A00537563636573732EB2
:10AB600020425420636F64652073657420746F20E5
:10AB7000272573272028616C776179732061203441
:10AB800020646967697420636F6465292E0A006216
:10AB900074636F6D6D616E64005265706C793A0A12
:10ABA00025730A00656570726F6D00626F61726473
:10ABB0006D6F64656C00626F6172646877636F6E5D
:10ABC0006669670063757272656E74726573697326
:10ABD000746F720073657269616C636F6D6D006C88
:10ABE00065667400726967687400736E0068656CEE
:10ABF0007000616870007374617475730061626FD6
:10AC00007574007363616E62757300636C6F736556
:10AC100000706172746F70656E00736574706F732D
:10AC2000007265737461727400636F6D6D62726936
:10AC30006467650077726200777277007265620000
:10AC400072657700466978656453697A6544786C03
:10AC5000436F6D6D616E6451756575650046697809
:10AC6000656453697A6544786C436F6D6D616E6499
:10AC700051756575655F627974657361727261792A
:10AC800000466978656453697A6544786C436F6DF2
:10AC90006D616E6451756575655F62696469726C3A
:10ACA000697374000A44554D50204C4953540A00AE
:10ACB0004865616420616464722025702C205461B1
:10ACC000696C20616464722025702C204974656D64
:10ACD00020636F756E742025642C2070747220645C
:10ACE00069666572656E63652025640A0041646467
:10ACF000722025702C20536572766F2049442025E0
:10AD0000640A00636C735F4D61696E426F617264C7
:10AD10005F696E697400FFFF000000000000000022
:10AD2000C9400000D5390000053A000000000000CD
:10AD30000000000000000000BD4200005141000082
:10AD4000794100008B410000D941000025420000FC
:10AD50006D420000BB4400006D4600000000000092
:10AD60000000000000000000195A0000CD4700005C
:10AD7000F5470000195A0000195A0000195A00003E
:10AD8000195A0000195A0000195A0000000000006A
:10AD900000000000010000000200000003000000AD
:10ADA000040000000600000007000000080000008A
:10ADB000090000000A0000000B0000000C00000069
:10ADC0000D0000000E0000000F0000001000000049
:10ADD0001100000012000000130000001400000029
:10ADE0001500000016000000180000001900000007
:10ADF0001A0000001B0000001C0000001D000000E5
:10AE00001E0000001F0000002000000021000000C4
:10AE100022000000230000002400000025000000A4
:10AE20002600000027000000280000002900000084
:10AE30002A0000002B0000002C0000002D00000064
:10AE40002E0000002F000000300000003100000044
:10AE50003200000033000000340000003500000024
:10AE60003600000037000000380000003900000004
:10AE70003A0000003B0000003C0000003D000000E4
:10AE80003E0000003F0000004000000041000000C4
:10AE900042000000430000004400000044000000A5
:10AEA0004500000046000000470000004800000088
:10AEB000490000004A0000004B0000004C00000068
:10AEC0004D0000004E0000004F0000005000000048
:10AED0005100000052000000530000005400000028
:10AEE0005500000056000000570000005800000008
:10AEF00058000000590000005A0000005B000000EC
:10AF00005C0000005D0000005E0000005F000000CB
:10AF100060000000610000006200000063000000AB
:10AF2000640000006500000066000000660000008C
:10AF30006700000068000000690000006A0000006F
:10AF40006B0000006C0000006D0000006E0000004F
:10AF50006F0000007000000071000000720000002F
:10AF60007200000073000000740000007500000013
:10AF700076000000770000007800000079000000F3
:10AF80007A0000007B0000007C0000007C000000D4
:10AF90007D0000007E0000007F00000080000000B7
:10AFA0008100000082000000830000008400000097
:10AFB0008500000086000000860000008700000079
:10AFC00088000000890000008A0000008B0000005B
:10AFD0008C0000008D0000008E0000008F0000003B
:10AFE0008F0000009000000091000000920000001F
:10AFF00093000000940000009500000096000000FF
:10B0000097000000970000009800000099000000E1
:10B010009A0000009B0000009C0000009D000000C2
:10B020009E0000009F0000009F000000A0000000A4
:10B03000A1000000A2000000A3000000A400000086
:10B04000A5000000A6000000A7000000A700000067
:10B05000A8000000A9000000AA000000AB0000004A
:10B06000AC000000AD000000AE000000AF0000002A
:10B07000AF000000B0000000B1000000B20000000E
:10B08000B3000000B4000000B5000000B6000000EE
:10B09000B6000000B7000000B8000000B9000000D2
:10B0A000BA000000BB000000BC000000BD000000B2
:10B0B000BE000000BE000000BF000000C000000095
:10B0C000C1000000C2000000C3000000C400000076
:10B0D000C5000000C5000000C6000000C700000059
:10B0E000C8000000C9000000CA000000CB0000003A
:10B0F000CC000000CD000000CD000000CE0000001C
:10B10000CF000000D0000000D1000000D2000000FD
:10B11000D3000000D4000000D4000000D5000000DF
:10B12000D6000000D7000000D8000000D9000000C1
:10B13000DA000000DB000000DC000000DC000000A2
:10B14000DD000000DE000000DF000000E000000085
:10B15000E1000000E2000000E3000000E400000065
:10B16000E4000000E5000000E6000000E700000049
:10B17000E8000000E9000000EA000000EB00000029
:10B18000EB000000EC000000ED000000EE0000000D
:10B19000EF000000F0000000F1000000F2000000ED
:10B1A000F3000000F3000000F4000000F5000000D0
:10B1B000F6000000F7000000F8000000F9000000B1
:10B1C000FA000000FB000000FC000000FC00000092
:10B1D000FD000000FE000000FF0000000001000074
:10B1E0000101000002010000030100000401000051
:10B1F0000401000005010000060100000701000035
:10B2000008010000090100000A0100000B01000014
:10B210000C0100000D0100000D0100000E010000F6
:10B220000F010000100100001101000012010000D8
:10B2300013010000140100001501000016010000B8
:10B24000170100001701000018010000190100009B
:10B250001A0100001B0100001C0100001D0100007C
:10B260001E0100001F01000020010000210100005C
:10B270002101000022010000230100002401000040
:10B280002501000026010000270100002801000020
:10B29000290100002A0100002B0100002C01000000
:10B2A0002D0100002D0100002E0100002F010000E3
:10B2B00030010000310100003201000033010000C4
:10B2C00034010000350100003601000037010000A4
:10B2D00038010000390100003A0100003B01000084
:10B2E0003B0100003C0100003D0100003E01000068
:10B2F0003F01000040010000410100004201000048
:10B300004301000044010000450100004601000027
:10B310004701000048010000490100004A01000007
:10B320004B0100004C0100004D0100004E010000E7
:10B330004F0100004F0100005001000051010000CA
:10B3400052010000530100005401000055010000AB
:10B35000560100005701000058010000590100008B
:10B360005A0100005B0100005C0100005D0100006B
:10B370005E0100005F01000060010000610100004B
:10B38000620100006301000064010000650100002B
:10B39000660100006701000068010000690100000B
:10B3A0006A0100006B0100006C0100006D010000EB
:10B3B0006E0100006F0100007001000071010000CB
:10B3C00072010000730100007401000075010000AB
:10B3D000760100007701000078010000790100008B
:10B3E0007A0100007B0100007C0100007D0100006B
:10B3F0007E0100007F01000080010000810100004B
:10B40000820100008301000084010000850100002A
:10B410008601000088010000890100008A01000007
:10B420008B0100008C0100008D0100008E010000E6
:10B430008F010000900100009101000092010000C6
:10B4400093010000940100009501000096010000A6
:10B4500097010000980100009A0100009B01000084
:10B460009C0100009D0100009E0100009F01000062
:10B47000A0010000A1010000A2010000A301000042
:10B48000A4010000A6010000A7010000A80100001F
:10B49000A9010000AA010000AB010000AC010000FE
:10B4A000AD010000AE010000B0010000B1010000DC
:10B4B000B2010000B3010000B4010000B5010000BA
:10B4C000B6010000B7010000B9010000BA01000098
:10B4D000BB010000BC010000BD010000BE01000076
:10B4E000C0010000C1010000C2010000C301000052
:10B4F000C4010000C5010000C7010000C801000030
:10B50000C9010000CA010000CB010000CC0100000D
:10B51000CE010000CF010000D0010000D1010000E9
:10B52000D2010000D4010000D5010000D6010000C6
:10B53000D7010000D8010000DA010000DB010000A3
:10B54000DC010000DD010000DF010000E00100007F
:10B55000E1010000E2010000E4010000E50100005B
:10B56000E6010000E7010000E9010000EA01000037
:10B57000EB010000EC010000EE010000EF01000013
:10B58000F0010000F2010000F3010000F4010000EE
:10B59000F5010000F7010000F8010000F9010000CA
:10B5A000FB010000FC010000FD010000FF010000A4
:10B5B000000200000102000003020000040200007B
:10B5C0000502000007020000080200000902000056
:10B5D0000B0200000C0200000D0200000F02000030
:10B5E000100200001202000013020000140200000A
:10B5F0001602000017020000190200001A020000E3
:10B600001B0200001D0200001E02000020020000BC
:10B610002102000023020000240200002602000094
:10B6200027020000280200002A0200002B0200006E
:10B630002D0200002E020000300200003102000046
:10B64000330200003402000036020000370200001E
:10B65000390200003A0200003C0200003E020000F5
:10B660003F020000410200004202000044020000CC
:10B670004502000047020000490200004A020000A3
:10B680004C0200004D0200004F0200005102000079
:10B69000520200005402000056020000570200004F
:10B6A000590200005B0200005C0200005E02000024
:10B6B00060020000610200006302000065020000F9
:10B6C00066020000680200006A0200006C020000CE
:10B6D0006D0200006F0200007102000073020000A2
:10B6E0007402000076020000780200007A02000076
:10B6F0007C0200007E0200007F0200008102000048
:10B700008302000085020000870200008902000019
:10B710008B0200008D0200008E02000090020000EB
:10B7200092020000940200009602000098020000BD
:10B730009A0200009C0200009E020000A00200008D
:10B74000A2020000A4020000A6020000A80200005D
:10B75000AB020000AD020000AF020000B102000029
:10B76000B3020000B5020000B7020000B9020000F9
:10B77000BC020000BE020000C0020000C2020000C5
:10B78000C4020000C7020000C9020000CB02000092
:10B79000CE020000D0020000D2020000D50200005C
:10B7A000D7020000D9020000DC020000DE02000027
:10B7B000E1020000E3020000E5020000E8020000F0
:10B7C000EA020000ED020000F0020000F2020000B8
:10B7D000F5020000F7020000FA020000FC0200007F
:10B7E000FF02000002030000050300000703000041
:10B7F0000A0300000D030000100300001203000004
:10B8000015030000180300001B0300001E030000C6
:10B810002103000024030000270300002A03000086
:10B820002D03000030030000330300003603000046
:10B83000390300003D030000400300004303000003
:10B84000460300004A0300004D03000050030000BF
:10B8500054030000570300005B0300005E03000078
:10B860006203000065030000690300006D0300002F
:10B870007103000074030000780300007C030000E3
:10B880008003000084030000880300008C03000094
:10B890009003000094030000980300009D03000043
:10B8A000A1030000A5030000AA030000AE030000EE
:10B8B000B3030000B8030000BC030000C103000094
:10B8C000C6030000CB030000D0030000D503000036
:10B8D000DA030000DF030000E5030000EA030000D4
:10B8E000EF030000F5030000FB030000000400006C
:10B8F000060400000C0400001204000019040000FB
:10B900001F040000250400002C0400003304000084
:10B910003A04000040040000480400004F04000006
:10B92000560400005E040000660400006E0400007F
:10B93000760400007E0400008704000090040000EC
:10B9400099040000A2040000AC040000B60400004A
:10B95000C0040000CA040000D5040000E004000098
:10B96000EC040000F80400000405000011050000CC
:10B970001E0500002C0500003A05000049050000E6
:10B9800059050000690500007A0500008C050000DB
:10B990009F050000B3050000C8050000DE0500009B
:10B9A0004D616C6C6F63206661696C656420666FC5
:10B9B000722025730A005061636B65743A20003071
:10B9C000784646203078464620307800454550522B
:10B9D0004F4D2077726974652064656E69656420D7
:10B9E000627920696E7465726E616C2070726F741A
:10B9F000656374696F6E2E204E72206F66207772B9
:10BA00006974657320617474656D70746564206910
:10BA10006E20746869732073657373696F6E3A2062
:10BA200000417474656D7074696E6720746F20775F
:10BA300072697465206120424954206F6E20612034
:10BA40006269746D61702062757420697427732057
:10BA50006F7574206F662072616E67653B20746835
:10BA60006520616C6C6F7765642072616E6765201C
:10BA7000697320307E372E00090AFFFFFFFFFFFFAA
:10BA8000FFFFFFFFFFFFFF0D00060807FFFF0E0F80
:10BA9000FF0CFFFFFFFFFFFF0B05050E08090D0C54
:10BAA00006070F04001303931A9217C5858486872F
:10BAB000C4FF6FF07F030370037813F0800FFBD097
:10BAC0007047FFFF4008FE4340A004404408FE4387
:10BAD00044A004400018FE4300C004403000FE4370
:10BAE000309004403400FE43349004401C18FE4360
:10BAF0001CC004401018FE4310C004400818FE4348
:10BB000008C004400C18FE430CC004400C10FE4357
:10BB10000CB004401010FE4310B004401810FE4357
:10BB200018B004401C10FE431CB004401410FE4327
:10BB300014B004400418FE4304C004400010FE4347
:10BB400000B004400008FE4300A004400408FE4387
:10BB500004A004400C08FE430CA004400808FE4367
:10BB600008A004401418FE4314C004401818FE43F3
:10BB700018C004400410FE4304B004400810FE4303
:10BB800008B004401400FE43149004404C08FE43E7
:10BB90004CA004400420FE4304D004402410FE4383
:10BBA00024B004402010FE4320B004402810FE437F
:10BBB00028B004402C10FE432CB004400020FE436B
:10BBC00000D004404808FE4348A004401000FE4353
:10BBD00010900440090AFFFFFFFFFFFFFFFFFFFF78
:10BBE000FFFFFF0D00060807FFFF0E0FFF0CFFFF12
:10BBF000FFFFFFFF0B05FFFF00000000000000003B
:10BC0000AD7D0000C57D0000957D00009D7D00009C
:10BC1000997D0000A17D0000397D00004B7D000072
:10BC20006B7D00006F7D0000757D0000857D00004C
:10BC3000A57D0000A97D0000097D0000157D0000A4
:10BC4000217D00002D7D0000D57D0000B97D000024
:10BC50000000000000000000B17E0000C97E00006E
:10BC6000997E0000A17E00009D7E0000A57E000060
:10BC70003D7E00004F7E00006F7E0000737E00005E
:10BC8000797E0000897E0000A97E0000AD7E000064
:10BC90000D7E0000197E0000257E0000317E000030
:10BCA000D97E0000BD7E0000000000000000000002
:10BCB000B57F0000CD7F00009D7F0000A57F0000C4
:10BCC000A17F0000A97F0000417F0000537F00009A
:10BCD000737F0000777F00007D7F00008D7F000074
:10BCE000AD7F0000B17F0000117F00001D7F0000CC
:10BCF000297F0000357F0000DD7F0000C17F00004C
:10BD00000D0AFFFFFFFFFFFF000000000000000022
:10BD1000078300000D830000F7820000FB82000013
:10BD2000FF820000038300000015191500010000C8
:10BD30007887FF1F1200000000020000A287FF1F8B
:10BD40004300000000030000FC87FF1F000000000C
:10BD5000010309048A87FF1F000000000203090491
:10BD6000E687FF1F00000000030309040088FF1F8F
:10BD700000000000000000000000000000000000C3
:10BD80004300FFFF1888FF1F0020202020202020D4
:10BD9000202028282828282020202020202020207B
:10BDA000202020202020202020881010101010108B
:10BDB00010101010101010101004040404040404D7
:10BDC0000404041010101010101041414141414171
:10BDD0000101010101010101010101010101010153
:10BDE0000101010110101010101042424242424263
:10BDF0000202020202020202020202020202020223
:10BE000002020202101010102000000000000000CA
:10BE10000000000000000000000000000000000022
:10BE20000000000000000000000000000000000012
:10BE30000000000000000000000000000000000002
:10BE400000000000000000000000000000000000F2
:10BE500000000000000000000000000000000000E2
:10BE600000000000000000000000000000000000D2
:10BE700000000000000000000000000000000000C2
:10BE8000000000000000000000FFFFFF00000000B5
:10BE900000000000000000000000000000000000A2
:10BEA0000000000000000000000000000000000092
:10BEB0000000000000000000000000000000000082
:10BEC0000000000000000000000000000000000072
:10BED0000000000000000000000000000000000062
:10BEE000000000000000000000000000232D302BA7
:10BEF0002000686C4C00656667454647003031326B
:10BF000033343536373839414243444546003031C1
:10BF1000323334353637383961626364656600FF21
:10BF2000F8B500BFF8BC08BC9E4670473504000059
:10BF3000554F0000F17D0000F57E0000F97F000004
:04BF40001983000061
:10BF440000000000010000000A0400000892FF1F26
:10BF540008000000FFFFFFFF120100020200004082
:10BF6400C016830400010102030118035400650094
:10BF740065006E00730079006400750069006E004E
:10BF84006F0009024300020100C0320904000001ED
:10BF9400020201000524001001052401010104240A
:10BFA4000206052406000107058203100040090467
:10BFB4000100020A00000007050302400000070513
:10BFC4008402400000001603550053004200200084
:10BFD400530065007200690061006C0004030904E9
:10BFE4000C0300000000000000000000000000003E
:10BFF4000000000000000000000000008CBE0000F3
:10C00400ACBE0000CCBE0000000000000000000038
:10C01400000000000000000080BD000000000000DF
:10C02400000000000000000000000000000000000C
:10C0340000000000000000000000000000000000FC
:10C0440000000000000000000000000000000000EC
:10C0540000000000000000001888FF1F88BD0000D9
:00000001FF
